:020000040000FA
:2000000000000000000000000000000000000000000000000000000000000000800044001C
:2000200002043E060000000000000000000000000000000000000000000000000000000076
:200040000000000000000000000000003E0B000000003E0B000000003E0B000000003E0B7C
:20006000000000003E0B000000003E0B000000003E0B000000003E0B000000003E0B000013
:2000800000003E0B000000003E0B000000003E0B000000003E0B000000003E0B00000000F3
:2000A0003E0B000000003E0B000000003E0B000000003E0B000000003E0B000000003E0B8A
:2000C000000000003E0B000000003E0B000000003E0B000000003E0B0000000000000000FC
:2000E00000000000000000000000000000000000000000003E0B000000003E0B000000006E
:200100003E0B000000003E0B000000003E0B000000003E0B000000003E0B000000003E0B29
:20012000000000003E0B000000003E0B000000003E0B000000003E0B000000003E0B000052
:2001400000003E0B000000003E0B000000003E0B000000003E0B000000003E0B0000000032
:200160003E0B000000003E0B000000003E0B000000003E0B000000003E0B000000003E0BC9
:200180001C0000000210000000043E0B00000000060F1C000000061100000000300F00005D
:2001A0000000340F00000000370F00000000380F000000003C0F000000003F0F00000000D6
:2001C000250F01000000260F000000002D0F010000002E0F000000000A10A01C02003E0124
:2001E000BA0130003E02AA0131003E02000000000A11000001000D14001800000B14210221
:2002000000000E0F060000000F0F03000000001000C810003E02410000002D1146000000AD
:200220002E11040002001F0FC2000200BE0602A000003E015C000200200645000000031105
:20024000C2000200BE06201002003E01C2000200BE06001002003E0116000000200700008F
:20026000DBB1090FBB0830003E02000000000B1100000200010F00010000020F2F0417001D
:200280003E01410000002E1104000200140F40000200180F000000001C0F40148285CF7048
:2002A00094FFFF00000E000000804F7604000200000F000000B20F7040000000011142007F
:2002C00000000211470000000411040002043E061C0000000E1100000000800000A0020004
:2002E0003E0103000000000700A002003E01050000002007002000883F7001000000020D41
:2003000000000080BE51600002003E0600A002003E0107000000200700000000DC0F0000AE
:200320000000DD0F002000883F7001000000020D000080EDBE51600002003E0600A00200A6
:200340003E01080000002007000000883F7004000000020DC2000204BE0600000000000059
:2003600000000000000000008081BE51600002003E0600A002003E010800000020070000B7
:2003800000883F7004000000020DC2000204BE060000000000000000000000000000808186
:2003A000BE51600002003E0600A002003E01080000002007000000883F7004000000020D2E
:2003C000C2000204BE06000000000000000000000000000080EDBE51600002003E0600A0CF
:2003E00002003E01D8FFFF00000700A002003E01D6FFFF00000700A002003E01DAFFFF006A
:20040000000700A002003E0107000000200700000000DC0F00000000DD0F0020008C3F7094
:2004200001000000020D000080EDBF51600002003E0600A002003E01D8FFFF00000700A02B
:2004400002003E01DFFFFF00000700A002003E01E6FFFF00000700A002003E016000020068
:2004600020060000008C3F7004000000020DC2000204BE060000000000000000000000007C
:20048000000080EDBF51600002003E06000000000D10000000000B11400000001F1142004E
:2004A00000002E11470000000F111C0000000E1100000000800004000200DB1200000000E8
:2004C0000D11000000043E0A00000081CF7D20128281DF7D00000000000000000000000054
:2004E0000000000000000000000000000000000000000000000000000000000000000000FC
:200500000000000000000000000000000000000000000000000000000000000000000000DB
:200520000000000000000000000000000000000000000000000000000000000000000000BB
:2005400000000000000000000000000000000000000000000000000000000000000000009B
:2005600000000000000000000000000000000000000000000000000000000000000000007B
:2005800000000000000000000000000000000000000000000000000000000000000000005B
:2005A00000000000000000000000000000000000000000000000000000000000000000003B
:2005C00000000000000000000000000000000000000000000000000000000000000000001B
:2005E0000000000000000000000000000000000000000000000000000000000000000000FB
:2006000000002A06400001000000000002000000000003000000000004000000000005005B
:0A06200000000000060000000000CA
:20062A000E0000000000ED0C00010200030102000206DB0FC940040F042008003E01F91618
:20064A000204BE06308C02000011000000000000B88C02000110010013003E0101800200CA
:20066A000110011008003E010180020000118D8C02000010001002003E011C0102000006D2
:20068A00318C020000102E8C02000410041008003E01140102000206DB0FC940040F04200D
:2006AA0008003E01F9160204BE06318C02000011000000000000B98C0200011001001300D4
:2006CA003E01018002000110011008003E0101800200001101800200001022EC020000119D
:2006EA002A380200001324EC020000112C3802000013918C02000010001002003E01360126
:20070A00020000068C9D020000100D661900040F004011003E01FEFF0000010F000141000E
:20072A003E0104C018003E01000040003E018C9D02000011E1FFFFFF0C0F0CA00D003E01A9
:20074A00BA8C02000110010013003E0123EC020000112B380200001324EC02000110011114
:20076A0008003E0124EC020001112C380200001300000000000F001002003E01A401020084
:20078A000006C7000000001000000020010F010004003E014B010200000601000000000F9A
:2007AA00001002003E0146010200000617A20200140F00000000340F1A000000680F0100DC
:2007CA0000001E0E0000000000994B0102003E06FAA10200140F00000000340F1D00000098
:2007EA00680F010000001E0E00000000009901000000000F001002003E01750102000006D3
:20080A0017A20200140F00000000340F18EC0200150F00000000350F203802001C0F0A00B0
:20082A000000680F030000001E0E000000003E59000000803E5B000000803F5925EC02002D
:20084A00150F2D3802001C0F02000000260F020000002D0F08000000680F030000001E0EB5
:20086A00000000003E5900000080BE5B000000807F5902800200150F08000000680F0200BD
:20088A0000001E0E000000003E59000000803E5BC60000000010FFCFFFFF010F01000400BB
:2008AA003E01C6000000001117A20200000F38000000001101000000000F390000000011AB
:2008CA001A000000000F3A0000000011C6000000001000300000010FA40102043E06011084
:2008EA0004003E01C60000000011FAA10200140F00000000340F0EEC0200150F00000000B1
:20090A00350F163802001C0F0A000000680F030000001E0E000000003E59000000803E5BAE
:20092A00000000803F5924EC0200150F2C3802001C0F02000000260F020000002D0F080051
:20094A000000680F030000001E0E000000003E5900000080BE5B000000807F5902800200DB
:20096A00150F08000000680F020000001E0E000000003E59000000803E5B000000003E5955
:20098A0022EC020000112A3802000013000000003E5924EC020000112C3802000013000082
:2009AA0000003E5923EC020000112B3802000013C60000000010FFCFFFFF010F0100040045
:2009CA003E01C60000000011FAA10200000F38000000001101000000000F390000000011A8
:2009EA001D000000000F3A0000000011C6000000001000300000010F011004003E01C60046
:200A0A000000001100000000000F35EC0200001136EC0200001137EC0200001138EC0200E7
:200A2A000011A5E70200140F00000000340F35EC0200150F00000000350F6BA102000810F6
:200A4A000C000000080D882804003E59001002003E01BA0102000006CC2C04003E010400CD
:200A6A000000000D153802001C0F000080163E59000000287F0400C8582A012900C8580079
:200A8A003E018C1808003E01000000843E5BF9E30200140F39EC0200150F6DA10200081091
:200AAA000C000000080D882804003E59001002003E01CA0102000006CC2C04003E0104005D
:200ACA000000000D153802001C0F000080163E59000000287F0400C8582A012900C8580019
:200AEA003E018C1808003E01000000843E5BF00A0000340F31A20200440F21AD020014104C
:200B0A00000000283F0421AD02001411C9A10200261035EC0200150F47EE0200160F000026
:200B2A000000360F6BA10200001004000000000D000000804F71000000803E5D00000000DC
:200B4A003E5B00000080BE59000001008014010202001A06000004008014E00102001A0606
:200B6A00000002008014020202003A0652EC0200160F00000000360F39EC0200150F6DA18C
:200B8A0002006810020000001E0E000000023E5B000000823E5D21AD0200011022AD020039
:200BAA00011113B80200011014B80200011105D90200011006D90200011147EE020001102F
:200BCA004BEE0200011148EE020001104CEE0200011149EE020001104DEE020001114AEE56
:200BEA00020001104EEE02000111000002008014FB0102003A0653EE0200011052EE02001E
:200C0A00011100000000010F53EE02000111000004008014010202003A0651EE0200011024
:200C2A0050EE0200011100000000010F51EE02000111000007002014928C020001100A007F
:200C4A000000000F012000003E013A0202000006F00A0000340F23AD0200440F13B80200A8
:200C6A001410000000283F0413B802001411CBA10200261000000000000F6CA102006810AF
:200C8A00010000001E0E00000080BE5900000000340F00000000000F012000003E011602BC
:200CAA000200200600000000000F340202003E0601000000000F012000003E011B020200E8
:200CCA00200622EC02000010340202003E0602000000000F012000003E012002020020068D
:200CEA0023EC02000010340202003E0603000000000F012000003E0125020200200624EC7C
:200D0A0002000010340202003E0604000000000F012000003E013002020020060EEC020072
:200D2A00140F25EC0200150F00000000350F378C02006810020000001E0E000000003E5909
:200D4A00000000803E5BCE0302003E0605000000000F012000003E01CE03020020060EECF2
:200D6A000200001025EC0200150F00000000350F378C02006810010000001E0E00000080F2
:200D8A003E5BCE0302003E064DEC02000410409402003E014DEC020004114EEC0200041095
:200DAA00409402003E014EEC0200041147EE0200100F00000000300F97A10200110F0000D4
:200DCA000000310FA7A10200120F00000000320FB7A10200130F00000000330F25EC02004C
:200DEA00150FEEED0200160F00000000360F19EE0200170F00000000370FC7A10200261069
:200E0A0000000000270FCBA102002D10000000003D0F003002001E0F000000003E0F0034BB
:200E2A0002001F0F000000003F0F4FEC02000310000000000F0F13B802000E106CA10200C2
:200E4A000D10F00A0000340F31A20200440F00000004FE5B000000003E5300A082003E5563
:200E6A00000000900F7010A102003E400000008A0F703FC02C003E01760202003006000005
:200E8A00008EEF71CC2C0422012901000000010D00C85822012900C858003E018C1808008C
:200EAA003E01040000008014760202003A060000808EFF71F00A0000340F23AD0200440FB7
:200ECA000000008AEF70CC2C04620129000080003E5710A102003E0101000000010D00C8B9
:200EEA005862012900C858003E018C1808003E01000000A87F04000000E87F04F00A00002A
:200F0A00340F23AD0200440F00008085EF700000008AEF70000000303F04000000874F7158
:200F2A0000000002FE5D77BE7F3F000F000080808F7080380E003E01812108003E018F02CA
:200F4A0002000006020000000C0F409402003E014C2C00003E0192020200040600004000B6
:200F6A00001416EE020001101F012C003E01920202043E0616EE0200011100000000040FA8
:200F8A00920202003E0640A402003E0192020200220600000000040F000000823E5D00005A
:200FAA0000843E5B0000008ABF70000000283F04000000843E59880413003E01000080006D
:200FCA00FE5F141108003E01000080803E5FF09F02003E01DF2100003E015902020024060B
:200FEA0018EE02000010009002003E0118EE02000011F00A0000340F23AD0200440F13B8B8
:20100A0002001410000000283F0413B802001411010000008014CE0302003A06100000008B
:20102A008014CE0302003A0600000000000F001002003E01810302040006F00A0000340FD2
:20104A0015CE0200440F01000000000F001002003E011A030204000602800200150F00001C
:20106A000000350F05D902001410000000283F0405D902001411C8A102002610F1FFFFFF1F
:20108A000C0FEDA1020003104FEC02000210000000000F0F6CA1020008102FC02C003E019A
:2010AA00CC020204300600000000040FF09F02003E018A9D020000100D661900040F004021
:2010CA0011003E01FEFF0000010F000141003E0104C018003E01000440003E018A9D020061
:2010EA00041114F001783E021CA00D003E01030413003E0100000082BE5900000000FE5BC1
:20110A00000000823E5B8F2400003E01D5020200040600000080BE59F09F02003E018F20BF
:20112A0000003E01BD02020024060400000080140B0302003A060800000080140B030200E7
:20114A003A06003402001F0FF00A0000340F07D90200440F25EC0200150FF00A0000360FF9
:20116A0015CE0200460F05D902001610F00A0000370F07D90200470FF7E3020017104FEC6F
:20118A0002000310000000000F0FB7A10200130F6CA102000D100000008EFF710000008AE2
:2011AA007F713FC02C003E01F20202043006882884003E5710A10206BE5D000000220129B2
:2011CA0001000000010D00C85822012900C858003E018C1808003E0100000000FE5B0810CF
:2011EA0008027F5F000000803E5B0000008A7F71000000283F04000000843E59000000F0F4
:20120A003F04F09F02003E01FD2000003E0107030200220600000006BE5D0000008A7F7186
:20122A00000000283F04000000863E59000000E03E04000000F03F04000000603F04000024
:20124A0000E87F04F09F02003E01FD2000003E01E70202000206F7E302001710CE03020420
:20126A003E06000000E83F04F7E30200171105D90200141025EC0200150F02000000020FA3
:20128A00000000000F0F6CA102000D1000000000BE5900008000FE5B011108003E010000B1
:2012AA0080803E5B000000303F04000000603F042F1F00003E01FD2000003E01CE030200B9
:2012CA002206100302003E0605D902001410000000283F0405D902001411C8A1020026106E
:2012EA00F1FFFFFF0C0FEDA1020003104FEC02000210000000000F0F6CA1020008100000A4
:20130A000000FE5B00000080BE59F09F02003E018F2400003E013C03020004062FC02C00AB
:20132A003E0137030204300600000000040FF09F02003E018A9D020000100D661900040F33
:20134A00004011003E01FEFF0000010F000141003E0104C018003E01000440003E018A9DA0
:20136A000200041114F001783E021CA00D003E01030413003E0100000082BE590000008213
:20138A003E5B8F2000003E019B0302000406230302003E06040000008014720302003A0657
:2013AA00080000008014720302003A06003402001F0FF00A0000340F07D90200440F25ECE9
:2013CA000200150FF00A0000360F15CE0200460F05D902001610F00A0000370F07D902003C
:2013EA00470FF7E3020017104FEC02000310000000000F0FB7A10200130F6CA102000D1074
:20140A0000000006BE5D0000008A7F71000000283F04000000863E59000000E03E0400007D
:20142A0000F03F04000000603F04000000E87F04F09F02003E01FD2000003E016E030200C2
:20144A0022060000008EFF710000008A7F713FC02C003E01640302043006882884003E570C
:20146A0010A10206BE5D00000022012901000000010D00C85822012900C858003E018C18C4
:20148A0008003E0100000000FE5B081008027F5F000000803E5B0000008A7F7100000028E7
:2014AA003F04000000843E59000000F03F04F09F02003E01FD2000003E014E03020002060A
:2014CA00F7E302001710CE0302043E06000000E83F04F7E30200171102000000020F0100A1
:2014EA0000000F0F6CA102000D1005D90200141025EC0200150F000000303F04000000608A
:20150A003F04FD2000003E01CE030200220600000000BE5900008000FE5B011108003E01DE
:20152A00000080803E5B2F1F00003E01770302003E0605D902001410000000283F0405D96E
:20154A0002001411C8A102002610F1FFFFFF0C0FEDA1020003104FEC0200021000000000BE
:20156A000F0F6CA102006810100000001E0E2FC02C003E019A030204300600000000040F3A
:20158A00F09F02003E018A9D020000100D661900040F004011003E01FEFF0000010F0001FB
:2015AA0041003E0104C018003E01000040003E018A9D02000011E1FFFFFF0C0F0CA00D001B
:2015CA003E01030413003E0100000082BE59040000008014C60302003A0608000000801491
:2015EA00C60302003A06003402001F0FF00A0000340F07D90200440F25EC0200150FF00ACF
:20160A000000360F15CE0200460F05D902001610F00A0000370F07D90200470FF7E30200E7
:20162A0017104FEC02000310000000000F0FB7A10200130F6CA102000D100000008EFF7165
:20164A000000008A7F713FC02C003E01B80302043006882884003E5710A10206BE5D000008
:20166A000022012901000000010D00C85822012900C858003E018C1808003E01000000004F
:20168A00FE5B081008027F5F000000803E5B0000008A7F71000000283F04000000843E59CE
:2016AA00000000F03F04F09F02003E01FD2000003E01AD0302000206F7E302001710CE0333
:2016CA0002043E06000000E83F04F7E30200171105D90200141025EC0200150F6CA102003D
:2016EA00681000000000BE59030000001E0E00008000FE5B01110800BE59000080803E5B7F
:20170A0001000000200F00000000340F00000000000F001002003E01DC030204000624ECF1
:20172A000200140F0F000000040F01000000000F001002003E01DC030204200602000000EA
:20174A00200F00000000000023EC0200140F23EC0200001160410000010F010070000111C6
:20176A0009000000000F009002003E0104000000000D000000003E5804910D003E011100DD
:20178A0010203E0200007000011100000000000F001002003E0135040200000601000000AB
:2017AA00000F001002003E01130402000006FAA10200150F00000000350F0EEC0200140F7C
:2017CA0000000000340F0A000000680F020000001E0E000000003E59000000803E5B24EC4D
:2017EA000200140F02000000260F08000000680F020000001E0E00000000BE59000000803F
:20180A003E5B02800200140F08000000680F020000001E0E000000003E59000000803E5B21
:20182A0022EC02000010000000803E5B24EC02000010000000803E5B23EC02000010000009
:20184A0000803E5BC60000000010FFFCFFFF010F010004003E01C60000000011FAA10200CE
:20186A00000F30000000001101000000000F3100000000111D000000000F3200000000114D
:20188A00C6000000001000030000010F011004003E01C60000000011350402003E0617A2F2
:2018AA000200150F00000000350F18EC0200140F00000000340F0A000000680F02000000C5
:2018CA001E0E000000003E59000000803E5B25EC0200140F02000000260F08000000680F36
:2018EA00020000001E0E00000000BE59000000803E5B02800200140F08000000680F020058
:20190A0000001E0E000000003E59000000803E5BC60000000010FFFCFFFF010F01000400FD
:20192A003E01C6000000001117A20200000F30000000001101000000000F3100000000112A
:20194A001A000000000F320000000011C6000000001000030000010F011004003E01C6000E
:20196A0000000011350402003E06B80B0000340F4B800200440F038C02001410FCFFFFFFF9
:20198A00260F000000303F04038C020014110DEC0200150F00000000350F948C0200261024
:2019AA00000000703F0400000000BE5B000000803E590DEC0200150F958C020026100000C2
:2019CA0000703F0400000000BE5B000000803E590DEC0200150F968C020026100000007031
:2019EA003F0400000000BE5B000000803E590DEC0200150F978C02002610000000703F043D
:201A0A0000000000BE5B000000803E59080000002B14100000002B14200000002B14000493
:201A2A0000002B14000000043E0A800000002B14008002007C101000000080146004020436
:201A4A003A0601000000200F7BA102002110F00A0000300F15CE0200400F640402043E069E
:201A6A0006D902001010C8A102002210F00A0000300F23AD0200400F14B802001010C7A10E
:201A8A000200221071A1020023107FEE0200001015B80200110F00000000310F000000997A
:201AAA000F73000000A10F746CA102006810060000001E0E000000890F71000000883E04EA
:201ACA0002000000000D000080003E54000080803E52000000103E04F00A0000300F31A2ED
:201AEA000200400F7FA102000010001002003E017C04020000064BEE0200101071A1020011
:201B0A006810020000001E0E000080003E50000080803E5280A102000010001002003E01F3
:201B2A008404020000064CEE0200101071A102006810020000001E0E000080003E500000E7
:201B4A0080803E5281A102000010001002003E018C04020000064DEE0200101071A102005D
:201B6A006810020000001E0E000080003E50000080803E5282A102000010001002003E0191
:201B8A0000000000000A4EEE0200101071A102006810020000001E0E000080003E5000000B
:201BAA0080803E52000000003E0A15BE0200110F00000000310FF00A0000300F31A2020000
:201BCA00400F01000000200F00000000210F7BA1020022102FEE0200120F00000000320F7B
:201BEA0000000000330F15BE0200130F78A10200001070A102000510051500003E017BA1DA
:201C0A0002000010502500003E012DEE02000511000080915F70000080801F710000808051
:201C2A003E54000000583E04000080801F71000080803E54000000583E04000080801F7122
:201C4A00000080803E54000000583E04000080801F71000080803E5415BE0200110F7FA117
:201C6A0002000010001002003E01BB04020000064BEE02001010000000103E040200000081
:201C8A00050D000080003E50000080803E52000000D83E04000000803F71000080880F70B9
:201CAA0080A102000010001002003E01C604020000064CEE02001010000000103E04020014
:201CCA000000050D000080003E50000080803E52000000D83E04000000803F7100008088F8
:201CEA000F7081A102000010001002003E01D104020000064DEE02001010000000103E044A
:201D0A0002000000050D000080003E50000080803E52000000D83E04000000803F710000BD
:201D2A0080880F7082A102000010001002003E01DC04020000064EEE020010100000001036
:201D4A003E0402000000050D000080003E50000080803E52040000008014000000003A0AA9
:201D6A0079A10200001070A102000510051500003E017BA102000010502500003E012EEEAE
:201D8A0002000511000080915F7033EE0200120F15C60200140F00000000340F00000000BA
:201DAA00350FF00A0000300F23AD0200400F14B802001010000000103E04000080980F73A1
:201DCA00000080A00F74C7A1020024106CA102006810090000001E0E000080880F71000074
:201DEA0000804F71000000803E540000808A0F7002000000050D000000003E5200000080DA
:201E0A003E5A000000183F04000000203E04000000003E0A01000000000F649502000011FF
:201E2A0003000000000F65950200001153480000000F66950200001141520000000F679523
:201E4A000200001143200000000F68950200001152440000000F69950200001159210000B3
:201E6A00000F6A9502000011200A0000000F6B950200001164950200000F78000000001158
:201E8A0001000000000F79000000001120080000000F7A0000000011879D0200000F68003F
:201EAA000000001101000000000F69000000001101000000000F6A0000000011F364040097
:201ECA00000F859D02000011F0000000001101000F00000FF40000000011F3200400000F69
:201EEA00F10000000011869D02000011002000000D14000800000D14000100000D14010013
:201F0A0000000A14005800000B1400000000000F5F8C02000011618C02000011638C020024
:201F2A000011658C02000011678C02000011698C020000116B8C020000116D8C020000115E
:201F4A006F8C02000011718C02000011A6050200BE06B6050200BE0600010000000F608C6B
:201F6A0002000011628C02000011648C02000011668C02000011688C020000116A8C02003C
:201F8A0000116C8C020000116E8C02000011708C02000011728C02000011A6050200BE067D
:201FAA00B6050200BE0600060000000F06000000010F011004003E01738C02000011758C04
:201FCA0002000011778C02000011798C020000117B8C020000117D8C020000117F8C020073
:201FEA000011818C02000011838C02000011A6050200BE06B6050200BE0600070000000F7C
:20200A0006000000010F011004003E01748C02000011768C02000011788C020000117A8C07
:20202A00020000117C8C020000117E8C02000011808C02000011828C02000011A60502005E
:20204A00BE06B6050200BE06ABC2A245010FBB8C0200011151480000000FA6050200BE0659
:20206A00B6050200BE06B6050200BE0651080000000FA6050200BE06C8000000680F02003A
:20208A0000001E0EB6050200BE0600000000000051070200BE0689150000010F878C0200A8
:2020AA00011100000000020F01420000000F010070000011000070000211888C0200021173
:2020CA0002420000000F010070000011000070000211898C02000211B6050200BE06000AE9
:2020EA000000000FA6050200BE06B6050200BE0609000000000F00A002003E018006000056
:20210A00030F80070000020F8A050200000600A002003E018D050200000600A002003E0118
:20212A0090050200000600A002003E0193050200000600A002003E0196050200000600A053
:20214A0002003E0199050200000600A002003E019C050200000600A002003E019F0502007D
:20216A000006A20502003E0623410000010F01007000011100007000031123410000010F73
:20218A0001007000011100007000021126410000010F01007000011100007000031126414A
:2021AA000000010F01007000011100007000021129410000010F0100700001110000700092
:2021CA00031129410000010F0100700001110000700002112C410000010F01007000011161
:2021EA000000700003112C410000010F010070000111000070000211008F0000000FA60585
:20220A000200BE06B6050200BE06000000003E0A20410000010F01007000011100007000C1
:20222A00001123410000010F01007000011100007000001126410000010F01007000011111
:20224A0000007000001129410000010F0100700001110000700000112C410000010F0100F7
:20226A0070000111000070000011000000003E0AB9050200BE06B9050200BE060000000001
:20228A003E0A0A800200031101000000030F338C02000311338C02000310301302003E010C
:2022AA00BC05020020060A8002000310000000003E0A0C800200140F00000000340F01004F
:2022CA000000240F11800200150F00000000350F868C0200001000A002003E01DD050200DD
:2022EA000206D40502002406FFFFFFFF000F68EC0200001169EC020000116AEC0200001184
:20230A00FF000000010F7AA102000010011104003E017AA102000111C08A0000040FD905B8
:20232A0002003E0600000000000F68EC0200001169EC020000116AEC02000011008A00007C
:20234A00040F05000000680F010000001E0E000000823E5B800602003E06FDFFFFFF040FC3
:20236A00BB8C0200001004910D003E0117EE02000010102100003E0100000000240A000064
:20238A000000000F17EE020000117DEE0200031000000000080F7DEE0200081100000000EF
:2023AA000F0F130000000C0F04000000020F05000000680F060000001E0E3FC02C003E019A
:2023CA00F20502041006F09F02003E010000000000008C082C003E01C22C00003E010000E4
:2023EA000000090F130000000C0F05000000680F060000001E0E3FC02C003E01FC0502046E
:20240A001006F09F02003E010000000000009C092C003E01C22C00003E016CA1020001106F
:20242A006EEC02000010012000003E01F2060200A0064FEC020001106FEC0200001001204A
:20244A0000003E01F2060200A0066BEC020003108A8C02000110101102003E010B06020089
:20246A00000611000000070F37032C003E01918C02000110101102003E01100602000006D0
:20248A0010000000070F37032C003E01008A0000040F381304003E0100410000010F0100EA
:2024AA0070000111000070000010000000803E5903410000010F01007000011100007000B2
:2024CA000010000000803E5906410000010F010070000111000070000010000000803E595A
:2024EA0009410000010F010070000111000070000010000000803E590C410000010F010000
:20250A0070000111000070000010000000803E590C800200140FC6ED0200160F000000000D
:20252A00360F00000000080F00000000070F000000000B0F120000000C0F040000000F0FB6
:20254A0005000000680F260000001E0E000000003E590C000000010F010104003E010400A7
:20256A000000020F122100003E013C06020004063C032C003E0187082C003E0170970200D3
:20258A003E013F0602043E06408A0000040F01000000009D008A0000040F00000000009DAE
:2025AA00709702003E01CF2C00003E0146060200240668EC020003116CEC020003103913F4
:2025CA0004003E01120000000C0F010000000B0F30000000010F010104003E0110000000D1
:2025EA00020F122100003E015206020004063C032C003E0180000000010F87082C003E01B6
:20260A00709702003E01540602043E06141404003E0101000000009D00000000009D709717
:20262A0002003E01CF2C00003E01000000823E5BB01B02003E015B060204200669EC02000A
:20264A00031101000000000F68EC02000311001002003E01D806020000066DEC0200001040
:20266A00000020008014620602003A06020000000F0F0F002C003E01000000048014680652
:20268A0002043A064FEE02000110101102003E01010000000F0F0F002C003E016D06020426
:2026AA0000066DEC02000011000000000000040000000F0F0F002C003E010000000180146D
:2026CA00710602003A06030000000F0F0F002C003E01010000008014750602003A06050045
:2026EA0000000F0F0F002C003E010200000080147B0602043A06928C020001100A000000A0
:20270A000C0F060000000F0F0F002C003E011C2100003E017F0602002006070000000F0FA8
:20272A000F002C003E016AEC0200001101000000000F001002003E01D80602000006EC1D5C
:20274A000200BE06B08C020000103E8002000110012100003E01940602002006AA8C02002F
:20276A000010418002000110012100003E01940602002006AB8C020002104080020001102A
:20278A00212100003E01940602002006AF8C020002103F8002000110212200003E01D8066B
:2027AA0002000006B08C020002103E8002000211AF8C020002103F8002000211AB8C020088
:2027CA000210408002000211AA8C02000210418002000211AA8C02000010001002003E014F
:2027EA00D8060200000602000000010F012100003E01B406020020060A000000000F928C5D
:20280A0002000011B08C0200001002000000010F012100003E01AB0602002006C506020430
:20282A003E0602000000001401000000001403000000010F012100003E01B10602002006CC
:20284A00C50602043E06020000002014010000000014C50602043E060200000000140100E2
:20286A0000002014AB8C0200001003000000010F102100003E01BB06020020060100000064
:20288A00000F928C02000011C50602003E0602000000010F102100003E01C306020020066A
:2028AA000A000000000F928C02000011C50602043E06020000002014010000002014000044
:2028CA000000000F928C02000011AF8C0200001000000000010F012100003E01CE0602001A
:2028EA00200601000000000F8A8C02000011D70602043E0600000000000F918C0200001109
:20290A0000000000010F8A8C0200011103000000010F012100003E01D70602040006010015
:20292A000000000F918C0200001101000000000F8A8C020000110000000000001180020082
:20294A00150F20410000010F010070000111000000003E5B00007000001123410000010FC7
:20296A00010070000111000000003E5B00007000001126410000010F0100700001110000B6
:20298A0000003E5B00007000001129410000010F010070000111000000003E5B000070000D
:2029AA0000112C410000010F010070000111000000003E5B0000700000117AA102000010B5
:2029CA00081004003E017AA102000011B6050200BE06000000003E0A00000000000F6CA17F
:2029EA00020001106EEC02000111101102003E0107070200000610A102003E0107070204CE
:202A0A0000060D000000070F07002C003E0110A102003E0107070204000609000000070FE6
:202A2A0007002C003E0110A102003E0107070204000605000000070F07002C003E0110A1D0
:202A4A0002003E0107070204000601000000070F07002C003E014FEC020003106FEC0200DB
:202A6A000311000000000F0F3FC02C003E010E07020030060C000000070F07002C003E01CF
:202A8A00F09F02003E013FC02C003E0113070200300608000000070F07002C003E01F09F81
:202AAA0002003E013FC02C003E0118070200300604000000070F07002C003E01F09F0200ED
:202ACA003E013FC02C003E011D070200300600000000070F07002C003E01F09F02003E018F
:202AEA006BEC0200001100000000000F6CA10200011004000000070F172100003E0150074B
:202B0A000200040610A102003E0138070204000611000000070F07002C003E0110A1020016
:202B2A003E013807020400060D000000070F07002C003E0110A102003E013807020400062F
:202B4A0009000000070F07002C003E0110A102003E0138070204000605000000070F07007B
:202B6A002C003E0110A102003E0138070204000601000000070F07002C003E013FC02C00EF
:202B8A003E013C070200300610000000070F07002C003E01F09F02003E013FC02C003E019F
:202BAA004107020030060C000000070F07002C003E01F09F02003E013FC02C003E01460770
:202BCA000200300608000000070F07002C003E01F09F02003E013FC02C003E014B07020095
:202BEA00300604000000070F07002C003E01F09F02003E013FC02C003E0150070200300640
:202C0A0000000000070F07002C003E016CEC02000011BB8C02000010B48C02000C107F077A
:202C2A000200BE06000000860F70DB0FC940000F7F070200BE062C8C0200001100000000A6
:202C4A00070F2F8C020007118E8C02000710701702003E016C07020000062C8C020000103F
:202C6A00000000000C0F308C02000C118F8C02006810010000001E0E0C1C08003E012D8C6A
:202C8A0002000C112C8C02000010000000000C0F318C02000C11908C0200681001000000B3
:202CAA001E0E0C1C08003E012E8C02000C11000000003E0ABB8C02000010B58C02000C1096
:202CCA007F070200BE06000000860F70DB0FC940000F7F070200BE062D8C0200001100007F
:202CEA000000070F308C02000711BB8C02000010B68C02000C107F070200BE060000008653
:202D0A000F70DB0FC940000F7F070200BE062E8C0200001100000000070F318C0200071122
:202D2A00000000003E0A000000400B0FC0408C830F700C0C13003E013C7059003E010C0C93
:202D4A0013003E013C7059003E010C0C13043E0A3C7059003E01070013003E0142800200FB
:202D6A0000114380020001114480020002114580020010114680020020114780020030119D
:202D8A00488002007C1100000000300F879D02000010000010103E02889D020001101011A4
:202DAA0000003E0111F802783E02889D020001114A800200011000FFFFFF020F12010400CC
:202DCA003E01101100003E010A0A0A0A020F122200003E01AF0702000006110802003E0285
:202DEA004A8002000111899D02000010009002003E01899D02000011108010003E02C20700
:202E0A000200300610FE01783E0210A102003E01000000901F70448D0200100F889D02007F
:202E2A000110000080803E4000000000010F889D0200011110040000010F01A000003E01AC
:202E4A00C20702000206899D02000010108010003E02B70702001006009002003E01889DB1
:202E6A000200011011F802783E02889D02000111B00702003E06899D0200001010FE01787D
:202E8A003E02000000901F70448D0200100F889D02000110000080803E4000000000000F12
:202EAA00899D02000011889D0200001101000000000F849D02000011879D0200000F6800B6
:202ECA000000001101000000000F69000000001101000000000F6A000000001100000000C2
:202EEA00000FF10000000011869D02000010F100000000114780020030104680020020107F
:202F0A00458002001010448002000210438002000110000000043E0A42800200001048802A
:202F2A0002007C10000000003E0A00000000011000700000020F121104003E0100000000B9
:202F4A00011102000000011000FCFFFF020F120104003E0121020000020F121104003E0147
:202F6A00020000000111348C0200100F01000000200F00000000300F80000000680F0100EB
:202F8A0000001E0E00000000009001000000000F81EE02000011B48C0200100F0100000077
:202FAA00200F00000000300F10000000680F010000001E0E00000000009002000000000F44
:202FCA0081EE020000110A000000000F368C0200001105420000010F01007000011100009D
:202FEA007000001109000000000F378C0200001106420000010F01007000011100900200EB
:20300A003E0100007000001100000000000F928C0200001100000000000F868C0200001172
:20302A0089150000000F878C020000110044AC45010FBB8C0200011100000000000F888CF0
:20304A0002000011898C020000111E000000000F7BA10200001104000000000F938C02009B
:20306A00001117000000000F948C0200001117000000000F958C0200001117000000000F5C
:20308A00968C0200001117000000000F978C02000011FF3F0000000F00000000010F0E9E8C
:2030AA00020000110F9E02000111109E02000111119E02000111129E02000111139E020036
:2030CA000011149E02000111159E02000111169E02000111179E0200011102000000000FA6
:2030EA0001430000010F01007000011114000000680F010000001E0E00007000001115435E
:20310A000000010F01007000011111000000680F010000001E0E00007000001100000000DC
:20312A00340F01000000240F00000000010F00010000000F1B0B0200BE0620010000000FD2
:20314A001B0B0200BE0640010000000F1B0B0200BE0660010000000F1B0B0200BE06800160
:20316A000000000F1B0B0200BE06A0010000000F1B0B0200BE06C0010000000F1B0B0200B6
:20318A00BE06E0010000000F1B0B0200BE0600020000000F1B0B0200BE0620020000000F57
:2031AA001B0B0200BE0640020000000F1B0B0200BE0660020000000F1B0B0200BE068002FD
:2031CA000000000F1B0B0200BE06A0020000000F1B0B0200BE06C0020000000F1B0B020054
:2031EA00BE06E0020000000F1B0B0200BE0600030000000F1B0B0200BE0620030000000FF4
:20320A001B0B0200BE0640030000000F1B0B0200BE0660030000000F1B0B0200BE06800399
:20322A000000000F1B0B0200BE06A0030000000F1B0B0200BE06C0030000000F1B0B0200F1
:20324A00BE06E0030000000F1B0B0200BE0600040000000F1B0B0200BE0620040000000F90
:20326A001B0B0200BE0640040000000F1B0B0200BE0660040000000F1B0B0200BE06800436
:20328A000000000F1B0B0200BE06A0040000000F1B0B0200BE06C0040000000F1B0B02008F
:2032AA00BE06E0040000000F1B0B0200BE0600050000000F1B0B0200BE0620050000000F2D
:2032CA001B0B0200BE0640050000000F1B0B0200BE0660050000000F1B0B0200BE068005D3
:2032EA000000000F1B0B0200BE0603420000000F01007000001101000000010F0000700072
:20330A00011104420000000F010070000011000070000111848C02000111858C02000111EF
:20332A000A420000000F01007000001101000000020F14000000680F010000001E0E0000DC
:20334A00700002111E420000000F01007000001101000000020F11000000680F0100000054
:20336A001E0E00007000021100000100000F3A8C0200140F00000000340F01000000240F22
:20338A0014000000680F010000001E0E000000803E594E8C0200140F11000000680F0100CC
:2033AA0000001E0E000000803E5901000000000F8A8C0200001101000000000F8B8C02005E
:2033CA00001100000000000F8C8C0200001100000000000F8D8C0200001100000000000F4E
:2033EA00918C0200001101000000000F8E8C0200001102000000000F8F8C02000011030014
:20340A000000000F908C020000110000C842000FB48C0200001100004843000FB58C02001B
:20342A00001100009643000FB68C020000110000003F000FB78C02000011CDCC4C3E000F5E
:20344A00B88C02000011CDCC4C3E000FB98C020000110000003F000FBA8C020000118E9DAF
:20346A000200140FCE9D0200150F00000000350F379E020000994B9E02000010000000805D
:20348A003E5B4C9E02000099609E02000010000000803E5B619E02000099759E020000101C
:2034AA00000000803E5B769E020000998A9E02000010000000803E5B8B9E020000999F9EE6
:2034CA0002000010000000803E5BA09E02000099B49E02000010000000803E5BB59E02000C
:2034EA000099C99E02000010000000803E5BCA9E02000099DE9E02000010000000803E5BED
:20350A00DF9E02000099F39E02000010000000803E5BF49E02000099089F020000100000E7
:20352A0000803E5B099F020000991D9F02000010000000803E5B1E9F02000099329F020013
:20354A000010000000803E5B339F02000099479F02000010000000803E5B489F0200009938
:20356A005C9F02000010000000803E5B5D9F02000099719F02000010000000803E5B729F38
:20358A0002000099869F02000010000000803E5B879F020000999B9F0200001000000080A9
:2035AA003E5B9C9F02000099B09F02000010000000803E5BB19F02000099C59F02000010B7
:2035CA00000000803E5BC69F02000099DA9F02000010000000803E5BDB9F02000099EF9F81
:2035EA0002000010000000803E5BF09F0200009904A002000010000000803E5B05A00200F6
:20360A00009919A002000010000000803E5B1AA0020000992EA002000010000000803E5BD5
:20362A002FA00200009943A002000010000000803E5B44A00200009958A00200001000007F
:20364A0000803E5B59A0020000996DA002000010000000803E5B6EA00200009982A00200AE
:20366A000010000000803E5B83A00200009997A002000010000000803E5B98A00200009924
:20368A00ACA002000010000000803E5BADA002000099C1A002000010000000803E5BC2A0D3
:2036AA0002000099D6A002000010000000803E5BD7A002000099EBA0020000100000008095
:2036CA003E5BECA00200009900A102000010000000803E5B01A10200009915A1020000104F
:2036EA00000000803E5B16A1020000992AA102000010000000803E5B2BA1020000993FA118
:20370A0002000010000000803E5B40A10200009954A102000010000000803E5B55A10200E0
:20372A00009969A102000010000000803E5B0100000000140200000000140400000020144E
:20374A0008000000001410000000001420000000001440000000001480000000201477A1CB
:20376A000200701101000000000F83A10200001102000000000F84A1020000110400000028
:20378A00000F85A10200001108000000000F86A10200001110000000000F87A1020000112C
:2037AA0020000000000F88A10200001140000000000F89A10200001180000000000F8AA14E
:2037CA000200001100010000000F8BA10200001100020000000F8CA1020000110004000028
:2037EA00000F8DA10200001100080000000F8EA10200001100100000000F8FA102000011B4
:20380A0000200000000F90A10200001100400000000F91A10200001100800000000F92A1D5
:20382A000200001100000000000F93A10200001194A10200001195A10200001196A102004B
:20384A00001101000000000F97A10200001198A10200001199A1020000119AA1020000110B
:20386A009BA1020000119CA1020000119DA1020000119EA1020000119FA102000011A0A168
:20388A0002000011A1A102000011A2A102000011A3A102000011A4A102000011A5A1020069
:2038AA000011A6A10200001120000000000F78A102000011A7A102000011A8A10200001181
:2038CA00A9A102000011AAA102000011ABA102000011ACA102000011ADA102000011AEA1B4
:2038EA0002000011AFA102000011B0A102000011B1A102000011B2A102000011B3A10200C3
:20390A000011B4A102000011B5A102000011B6A10200001179A102000011B7A102000011B9
:20392A00B8A102000011B9A102000011BAA102000011BBA102000011BCA102000011BDA1F9
:20394A0002000011BEA102000011BFA102000011C0A102000011C1A102000011C2A1020017
:20396A000011C3A102000011C4A102000011C5A102000011C6A10200001140000000000FFB
:20398A0070A10200001120000000000F71A10200001170A1020000107BA102000110012230
:2039AA0000003E017FEE0200021120A202003E017EEE0200021171A10200001000A00200F2
:2039CA003E0180EE0200001101000000000F6BA102000011F00A0000000FC9A10200001168
:2039EA0001000000000F7FA10200001100000000000F80A10200001181A10200001182A1DF
:203A0A000200001101000000000F6CA102000011FEFFFFFF000F76A1020000110000000025
:203A2A00000F001002003E01B0090200000601000000000F001002003E01B0090200200619
:203A4A00FFFFFFFF000F76A10200001100040000000FCBA102000011CAA102000011F00A1D
:203A6A000000000FC7A102000011F00A0000000FC8A10200001101000000000F6DA102000D
:203A8A0000110000803E000FECA102000011CDCCCC3D000FEDA1020000110AD7233C000FFD
:203AAA00EAA1020000116F12833A010FEBA102000111010013003E010000803F010F10211D
:203ACA0008003E0150EC02000111DAED0200100F00000000300F01000000200F14000000DA
:203AEA00680F010000001E0E000080803E50A5E70200100FBC000000680F010000001E0E7D
:203B0A0000000000009001000000000FA5E70200001115000000000FA6E702000011000098
:203B2A00803F000FA7E702000011F9E30200100F00000000300F01000000200FAC030000F1
:203B4A00680F010000001E0E000000000090F9E30200100F02000000000F0000803F010F4A
:203B6A0010000000680F040000001E0E010000000090000000803E50000080803E500090C7
:203B8A0002003E01C6ED0200100F14000000680F010000001E0E000000000090B80B0000FB
:203BAA00340F4B800200440F038C0200141101000000240FB80B0000680F010000001E0E47
:203BCA00000000000099000001002014000002002014000004002014000008000014000083
:203BEA001000001400000000000F7AA10200001105000000000F73A10200001172A102000A
:203C0A0000110B100000000F358C0200001104000000000FAC8C0200001109000000000F15
:203C2A00AD8C020000110A000000000FAE8C020000110A000000000F368C020000110900D1
:203C4A000000000F378C0200001167000000000FB38C0200001100000080AF77000000C047
:203C6A00010F010104003E0111E200783E02B18C0200011100000030010F010104003E0164
:203C8A0011E400783E02B28C0200011101000000010FA98C0200011100002000201400006D
:203CAA0040002014000080002014000000012014000000022014000000042014000000002F
:203CCA00000F4DEC020000114EEC02000011C4ED02000011C5ED0200001116EE0200001192
:203CEA004FEE0200001118EE0200001168EE0200001174A10200001175A10200001151EE58
:203D0A000200001153EE020000116DEC0200001117EE020000116CA1020001106EEC020032
:203D2A000111101102003E013B0A0200000610A102003E013B0A020400060D000000070F52
:203D4A0007002C003E0110A102003E013B0A0204000609000000070F07002C003E0110A162
:203D6A0002003E013B0A0204000605000000070F07002C003E0110A102003E013B0A0204DD
:203D8A00000601000000070F07002C003E014FEC020003106FEC02000311000000000F0FAB
:203DAA003FC02C003E01420A020030060C000000070F07002C003E01F09F02003E013FC0A8
:203DCA002C003E01470A0200300608000000070F07002C003E01F09F02003E013FC02C005A
:203DEA003E014C0A0200300604000000070F07002C003E01F09F02003E013FC02C003E0126
:203E0A00510A0200300600000000070F07002C003E01F09F02003E016BEC02000011000043
:203E2A000000000F6CA10200011004000000070F172100003E01840A0200040610A102006B
:203E4A003E016C0A0204000611000000070F07002C003E0110A102003E016C0A020400068A
:203E6A000D000000070F07002C003E0110A102003E016C0A0204000609000000070F070009
:203E8A002C003E0110A102003E016C0A0204000605000000070F07002C003E0110A10200F9
:203EAA003E016C0A0204000601000000070F07002C003E013FC02C003E01700A0200300692
:203ECA0010000000070F07002C003E01F09F02003E013FC02C003E01750A020030060C0043
:203EEA000000070F07002C003E01F09F02003E013FC02C003E017A0A020030060800000032
:203F0A00070F07002C003E01F09F02003E013FC02C003E017F0A0200300604000000070FFA
:203F2A0007002C003E01F09F02003E013FC02C003E01840A0200300600000000070F0700E8
:203F4A002C003E016CEC0200001176A1020001104FEC02000111EAA102000010EBA10200DD
:203F6A000110010013003E010000803F010F102108003E0150EC02000111DAED0200100F54
:203F8A0000000000300F01000000200F14000000680F010000001E0E000080803E50F00A68
:203FAA000000300F31A20200400F21AD02001011F00A0000680F010000001E0E0000000005
:203FCA000090F00A0000300F23AD0200400F13B802001011F00A0000680F010000001E0E61
:203FEA0000000000009000A00000300F00604200400F000043001011F00A0000680F010081
:20400A0000001E0E00000000009000A00000300F02004300400F02A043001011F00A000067
:20402A00680F010000001E0E000000000090F00A0000300F07D90200400FF7E302001011DB
:20404A00F00A0000680F010000001E0E000000000090F00A0000300F15CE0200400F05D9DD
:20406A0002001011F00A0000680F010000001E0E0000000000900DEC0200140F00000000C7
:20408A00340F01000000240F40000000680F010000001E0E000000000099EEED0200100F26
:2040AA0000000000300F01000000200F14000000680F010000001E0E00000000009019EE38
:2040CA000200100F6F12833A000F14000000680F010000001E0E000000803E5002EE0200B0
:2040EA00100F14000000680F010000001E0E000000000090EAA10200001070EC0200100F35
:20410A00A0000000680F010000001E0E000000803E50EAA1020000100000803E010F0100D7
:20412A0013003E0110ED0200100FA0000000680F010000001E0E000000803E500030020081
:20414A00180F00000000380F01000000280F00000000080F66EC02000010001002003E01E3
:20416A00E90A0200000600040000680F010000001E0E000000843F5000340200180F000022
:20418A000000380F01000000280F00000000080F00040000680F010000001E0E0000008453
:2041AA003F5001000000000F66EC0200001100000000380F00004200180F01000000280F09
:2041CA0017B7D138080F67EC02000010001002003E010E0B0200000600600000680F010038
:2041EA0000001E0E000000843F5000004200180F00004200190F00000000390FCAA10200EE
:20420A002910800000002A0F00000000000F00000000040F6DA1020005106CA1020002103A
:20422A0000000000010F7BA102006810010000001E0E000000803F50000000487E040000C8
:20424A00008C9F71109102003E01122300003E01FF0A02000206000000507E04000000502D
:20426A007E04000000507E04000000507E04409402003E01452600003E01FE0A020002063D
:20428A0001000000000F67EC0200001155380200180F00000000000F00060000680F01005B
:2042AA0000001E0E000000803F50553E0200180F00000000000F00060000680F0100000070
:2042CA001E0E000000803F50000000003E0A0E9E0200140F0100700000110A000000680F7D
:2042EA00030000001E0E000000003E59000070000011000070000111000000003E0A448DD2
:20430A00020002100000FFFF010F210204003E0122F002783E0243310000010F1221000088
:20432A003E012C0B0200000641430000010FCE1502002006458D020001108CEE02000111E3
:20434A00FF000000020F120204003E0147000000030F232200003E01FC1002002206414454
:20436A005021020F212200003E01430B02002006468D02000110101102003E013B0B020029
:20438A0000060100000000143C0B02003E06010000002014478D02000110101102003E01ED
:2043AA00410B02000006020000000014420B02003E06020000002014D81502003E06414C00
:2043CA004721020F212200003E01650B02002006468D02000110EAA102000111478D0200E5
:2043EA000110101102003E014D0B020000064000000000144E0B02003E0640000000201479
:20440A00488D02000110EBA102000111498D02000110101102003E01550B02000006200037
:20442A0000000014560B02003E062000000020144A8D0200011072A1020001114B8D020078
:20444A000110101102003E015D0B020000062000000000145E0B02003E06800000002014D8
:20446A00EAA102000010EBA102000110010013003E010000803F010F102108003E0150EC20
:20448A0002000111D81502003E0641534421020F212200003E016F0B02002006468D0200C8
:2044AA00011076A1020001114FEC02000210D81502043E06121204003E014FEC0200021179
:2044CA00D81502003E0642415544020F212200003E018A0B02002006468D020001108025A8
:2044EA000000020F122200003E01780B02002006BB200000000F860B02003E06004B000077
:20450A00020F122200003E017D0B02002006CC200000000F860B02003E0600E10000020F99
:20452A00122200003E01820B0200200688200000000F860B02003E0600C20100020F1222B3
:20454A0000003E01760B0200200666200000000F00420000010F010070000111000070008F
:20456A000011CE1502003E0643415421020F212200003E012A0C02002006468D0200011027
:20458A00478D0200021010A102003E01980B02002006738C02000110C0FFFFFF000F01018C
:2045AA0004003E01121104003E01738C0200011120410000000F260C02003E0610A102009A
:2045CA003E01A10B02002006748C02000110C0FFFFFF000F010104003E01121104003E0134
:2045EA00748C0200011120410000000F260C02003E0610A102003E01AA0B02002006758CE5
:20460A0002000110C0FFFFFF000F010104003E01121104003E01758C02000111234100008D
:20462A00000F260C02003E0610A102003E01B30B02002006768C02000110C0FFFFFF000F30
:20464A00010104003E01121104003E01768C0200011123410000000F260C02003E0610A1F3
:20466A0002003E01BC0B02002006778C02000110C0FFFFFF000F010104003E0112110400B2
:20468A003E01778C0200011126410000000F260C02003E0610A102003E01C50B02002006E2
:2046AA00788C02000110C0FFFFFF000F010104003E01121104003E01788C020001112641E3
:2046CA000000000F260C02003E0610A102003E01CE0B02002006798C02000110C0FFFFFF81
:2046EA00000F010104003E01121104003E01798C0200011129410000000F260C02003E06EC
:20470A0010A102003E01D70B020020067A8C02000110C0FFFFFF000F010104003E01121146
:20472A0004003E017A8C0200011129410000000F260C02003E0610A102003E01E00B020042
:20474A0020067B8C02000110C0FFFFFF000F010104003E01121104003E017B8C020001117D
:20476A002C410000000F260C02003E0610A102003E01E90B020020067C8C02000110C0FF53
:20478A00FFFF000F010104003E01121104003E017C8C020001112C410000000F260C02008B
:2047AA003E0610A102003E01F20B020020067D8C02000110C0FFFFFF000F010104003E0167
:2047CA00121104003E017D8C020001112F410000000F260C02003E0610A102003E01FB0B5D
:2047EA00020020067E8C02000110C0FFFFFF000F010104003E01121104003E017E8C0200E7
:20480A0001112F410000000F260C02003E0610A102003E01040C020020067F8C020001103D
:20482A00C0FFFFFF000F010104003E01121104003E017F8C0200011132410000000F260C24
:20484A0002003E0610A102003E010D0C02002006808C02000110C0FFFFFF000F01010400E4
:20486A003E01121104003E01808C0200011132410000000F260C02003E0610A102003E017D
:20488A00160C02002006818C02000110C0FFFFFF000F010104003E01121104003E01818C20
:2048AA000200011135410000000F260C02003E0610A102003E011F0C02002006828C020088
:2048CA000110C0FFFFFF000F010104003E01121104003E01828C0200011135410000000F9F
:2048EA00260C02003E06838C02000110C0FFFFFF000F010104003E01121104003E01838C8E
:20490A000200011138410000000F260C02003E06010070000011000070000111B6050200B8
:20492A00BE06D81502003E0643414C3F020F212200003E013F0C0200200601000000240F2D
:20494A0000000000340FEAA10200140F64950200110F00000000310F04000000210F0000CB
:20496A0000483E0401000000210F10000000080F809002003E0165950200001104000000E9
:20498A00080D000080007E58000080807E5211F000783E02000080807E52D1150200BE069D
:2049AA00C21502003E0643414E21020F212200003E015D0C02002006468D0200110F0000C4
:2049CA000000310F01000000210F6AA10200140F00000000340F80000000680F02000000F0
:2049EA001E0E000000007E52000000807E58EAA10200140F00000000340F10000000680FE1
:204A0A00020000001E0E000000007E52000000807E5814170200BE0601000000010F328C78
:204A2A000200011100430000000F01007000001100007000011100100000010F00420000A0
:204A4A00000F010070000011000070000111F9090200BE06D81502003E064341583F020F12
:204A6A00212200003E01730C0200200677A10200701101000000240F00000000340F6AA1E6
:204A8A000200140F64950200110F00000000310F04000000210F000000483E0401000000CD
:204AAA00210F80000000080F809002003E0165950200001104000000080D000080007E5858
:204ACA00000080807E5211F000783E02000080807E52D1150200BE06C21502003E06434225
:204AEA004C3F020F212200003E01880C0200200601000000240F00000000340FB48C020019
:204B0A00140F64950200110F00000000310F04000000210F000000483E0401000000210F1E
:204B2A0010000000080F809002003E0165950200001104000000080D000080007E58000077
:204B4A0080807E5211F000783E02000080807E52D1150200BE06C21502003E064342583F0D
:204B6A00020F212200003E019D0C0200200601000000240F00000000340F348C0200140F6B
:204B8A0064950200110F00000000310F04000000210F000000483E0401000000210F800041
:204BAA000000080F809002003E0165950200001104000000080D000080007E580000808007
:204BCA007E5211F000783E02000080807E52D1150200BE06C21502003E0643424E21020FA4
:204BEA00212200003E01B50C0200200600430000000F01007000001100000000000F00005D
:204C0A0070000011328C02000011468D0200110F00000000310F01000000210FC48C020080
:204C2A00140F00000000340F80000000680F020000001E0E000000007E52000000807E58B9
:204C4A00B48C0200140F00000000340F10000000680F020000001E0E000000007E5200001D
:204C6A0000807E58D81502003E0643474E21020F212200003E01700D02002006468D02009B
:204C8A000110478D0200021010A102003E01C30C020020065F8C02000110F0FFFFFF000F2E
:204CAA00010104003E01121104003E015F8C0200011120410000000F6C0D02003E0610A160
:204CCA0002003E01CC0C02002006608C02000110F0FFFFFF000F010104003E011211040022
:204CEA003E01608C0200011120410000000F6C0D02003E0610A102003E01D50C0200200641
:204D0A00618C02000110F0FFFFFF000F010104003E01121104003E01618C0200011123417D
:204D2A000000000F6C0D02003E0610A102003E01DE0C02002006628C02000110F0FFFFFFA9
:204D4A00000F010104003E01121104003E01628C0200011123410000000F6C0D02003E065B
:204D6A0010A102003E01E70C02002006638C02000110F0FFFFFF000F010104003E011211B6
:204D8A0004003E01638C0200011126410000000F6C0D02003E0610A102003E01F00C02009E
:204DAA002006648C02000110F0FFFFFF000F010104003E01121104003E01648C0200011115
:204DCA0026410000000F6C0D02003E0610A102003E01F90C02002006658C02000110F0FF82
:204DEA00FFFF000F010104003E01121104003E01658C0200011129410000000F6C0D0200F8
:204E0A003E0610A102003E01020D02002006668C02000110F0FFFFFF000F010104003E01D5
:204E2A00121104003E01668C0200011129410000000F6C0D02003E0610A102003E010B0DBA
:204E4A0002002006678C02000110F0FFFFFF000F010104003E01121104003E01678C02007E
:204E6A0001112C410000000F6C0D02003E0610A102003E01140D02002006688C0200011099
:204E8A00F0FFFFFF000F010104003E01121104003E01688C020001112C410000000F6C0D64
:204EAA0002003E0610A102003E011D0D02002006698C02000110F0FFFFFF000F0101040054
:204ECA003E01121104003E01698C020001112F410000000F6C0D02003E0610A102003E01EA
:204EEA00260D020020066A8C02000110F0FFFFFF000F010104003E01121104003E016A8CA7
:204F0A00020001112F410000000F6C0D02003E0610A102003E012F0D020020066B8C0200E6
:204F2A000110F0FFFFFF000F010104003E01121104003E016B8C0200011132410000000F22
:204F4A006C0D02003E0610A102003E01380D020020066C8C02000110F0FFFFFF000F010120
:204F6A0004003E01121104003E016C8C0200011132410000000F6C0D02003E0610A102007E
:204F8A003E01410D020020066D8C02000110F0FFFFFF000F010104003E01121104003E019F
:204FAA006D8C0200011135410000000F6C0D02003E0610A102003E014A0D020020066E8C2B
:204FCA0002000110F0FFFFFF000F010104003E01121104003E016E8C020001113541000089
:204FEA00000F6C0D02003E0610A102003E01530D020020066F8C02000110F0FFFFFF000F55
:20500A00010104003E01121104003E016F8C0200011138410000000F6C0D02003E0610A1D4
:20502A0002003E015C0D02002006708C02000110F0FFFFFF000F010104003E01121104001D
:20504A003E01708C0200011138410000000F6C0D02003E0610A102003E01650D0200200624
:20506A00718C02000110F0FFFFFF000F010104003E01121104003E01718C020001113B41E2
:20508A000000000F6C0D02003E06728C02000110F0FFFFFF000F010104003E0112110400BF
:2050AA003E01728C020001113B410000000F6C0D02003E0601007000001100007000011147
:2050CA00B6050200BE06D81502003E06434E5221020F212200003E01E00D02002006004323
:2050EA000000000F01007000001100000000000F000070000011328C020000110042000072
:20510A00000F01007000001100100000000F00007000001100000000000F66EC02000011E0
:20512A0067EC02000011F9090200BE0601000000240F00000000340F00005000150F00004C
:20514A000000350F00000000380F01000000280F000000003E5B000010103E02A5000000E4
:20516A00030F032000003E01B40D02002006C48C0200140F80000000680FBC0D0200BE06CD
:20518A00B48C0200140F10000000680FBC0D0200BE066AA10200140F80000000680FBC0D9A
:2051AA000200BE06EAA10200140F10000000680FBC0D0200BE0600004200180F0060000090
:2051CA00680FCE0D0200BE0600300200180F00040000680FCE0D0200BE0600340200180FDB
:2051EA0000040000680FCE0D0200BE06A5E70200140FBC000000680FBC0D0200BE06F9E33A
:20520A000200140FAC030000680FBC0D0200BE0600000000000F66EC0200001167EC0200E1
:20522A00001114170200BE0601000000010F328C0200011100430000000F010070000011AB
:20524A0000007000011100100000010F00420000000F010070000011000070000111D81560
:20526A0002003E0601000000010F328C0200011100430000000F01007000001100007000B7
:20528A000111434E5621010F8CEE02000111D81502003E06100000001E0E000000003E5B44
:2052AA00000010103E0210F802783E02000000003E5B000010103E02101100003E0111F860
:2052CA0002783E02000000003E5B000010103E02101100003E0111F802783E0200000000EE
:2052EA003E5B000010103E02101100003E0111F802783E02000080803E59000000003E0AA9
:20530A00100000001E0E000000003E5B000010103E0210F802783E02000000003E5B0000F3
:20532A0010103E02101100003E0111F802783E02000000003E5B000010103E0210110000C6
:20534A003E0111F802783E02000000003E5B000010103E02101100003E0111F802783E0225
:20536A00000080803F50000000003E0A434E5321020F212200003E014B0E02002006AA0089
:20538A000000000F55000000010F80000000020F10000000030F555550000011AA2A5000AD
:2053AA000111555550000211555550000011AA2A500001115555500003110A00000000006B
:2053CA000300ED0D02000E00000000003900F00D0200000050000B10000050000C10BC2BC0
:2053EA0000003E01F00D0200200601000000240F00000000340F00005000150F0000000054
:20540A00350F00000000250FAA000000000F55000000010FA0000000020FA5000000030F84
:20542A003F0E0200BE06000000603F04348C0200140F80000000680F1D0E0200BE06B48C9F
:20544A000200140F10000000680F1D0E0200BE066AA10200140F80000000680F1D0E020051
:20546A00BE06EAA10200140F10000000680F1D0E0200BE0600000000380F00004200180F86
:20548A0001000000280F00600000680F2E0E0200BE0600300200180F00040000680F2E0EE1
:2054AA000200BE0600340200180F00040000680F2E0E0200BE06A5E70200140FBC000000D5
:2054CA00680F1D0E0200BE06F9E30200140FAC030000680F1D0E0200BE06D81502003E060F
:2054EA000F0000001E0E000080013E593F0E0200BE06000000603F0433F800783E023F0E69
:20550A000200BE06000000603F0433F800783E023F0E0200BE06000000603F0433F80078DC
:20552A003E023F0E0200BE060A00000000000300290E02000E00000000000E002C0E020070
:20554A00000000603F04000000003E0A0F0000001E0E000080013F503F0E0200BE060000F8
:20556A0000603F0433F800783E023F0E0200BE06000000603F0433F800783E023F0E0200B3
:20558A00BE06000000603F0433F800783E023F0E0200BE060A000000000003003A0E02004D
:2055AA000E0000000000B00F3D0E0200000000603F04000000003E0A555550000011AA2AFD
:2055CA0050000111555550000211000080817E5B0000000000000000000000000000000276
:2055EA007E5B000000000000000080027E5B452400003E01450E02002006000000003E0A02
:20560A0044415421020F212200003E018E0E0200200601020000000F659502000011468D3D
:20562A0002000210938C0200021120A102003E01560E0200200600020000030F5B0E02000B
:20564A003E0610A102003E015A0E0200200600010000030F5B0E02003E0680000000030F26
:20566A00478D02000410488D02000510498D020006104A8D02000710B80B0000340F4B809B
:20568A000200440F04000000240F64950200110F00000000310F000000603E040100000076
:2056AA00210F401402003E016E0E02000006038C0200141004000000030D000080003E59B7
:2056CA00000080807E5211F000783E02000080807E52501502003E01770E02000006038CA5
:2056EA0002001410000000083F0404000000030D000080003E59000080807E5211F00078BB
:20570A003E02000080807E52601602003E01810E02000006038C02001410000000083F0421
:20572A00000000083F0404000000030D000080003E59000080807E5211F000783E02000060
:20574A0080807E52701702003E018C0E02000006038C02001410000000083F0400000008FD
:20576A003F04000000083F0404000000030D000080003E59000080807E5211F000783E02DD
:20578A00000080807E52D1150200BE06C21502003E0644535221020F212200003E01A20E19
:2057AA0002002006468D02000110478D0200021010A102003E01000000921F7000000000D6
:2057CA00340F948C0200140F000000203F04000000813E59B80B0000340F4B800200440F96
:2057EA00038C02001410000000203F0404000000240F00020000680F010000001E0E0000AA
:20580A0000000099D81502003E0645424321020F212200003E01CE0E02002006468D02005B
:20582A00001083A102000011478D0200001084A102000011488D0200001085A102000011D9
:20584A00498D0200001086A1020000114A8D0200001087A1020000114B8D0200001088A1E5
:20586A00020000114C8D0200001089A1020000114D8D020000108AA1020000114E8D0200DC
:20588A0000108BA1020000114F8D020000108CA102000011508D020000108DA10200001151
:2058AA00518D020000108EA102000011528D020000108FA102000011538D0200001090A155
:2058CA0002000011548D0200001091A102000011558D0200001092A102000011568D020054
:2058EA00001093A102000011578D0200001094A102000011588D0200001095A102000011C9
:20590A00D81502043E06598D0200001096A10200001146454E21020F212200003E01DC0E8D
:20592A0002002006468D0200011003420000000F010070000011000070000111848C0200E5
:20594A000111478D0200011004420000000F010070000011000070000111858C02000111C6
:20596A00D81502003E06464C5421020F212200003E01BD100200200600000000010F328C8D
:20598A000200011100430000000F010070000011000070000111468D02000110101102008A
:2059AA003E01DE0F02002006478D02000010488D02000210001102003E01800F02000006D1
:2059CA0010A102003E01F00E0200200600010000040F01430000050F4C0F02003E0610A1E7
:2059EA0002003E01F50E0200200620010000040F02430000050F4C0F02003E0610A1020050
:205A0A003E01FA0E0200200640010000040F03430000050F4C0F02003E0610A102003E01CC
:205A2A00FF0E0200200660010000040F04430000050F4C0F02003E0610A102003E01040FB2
:205A4A000200200680010000040F05430000050F4C0F02003E0610A102003E01090F020077
:205A6A002006A0010000040F06430000050F4C0F02003E0610A102003E010E0F020020060D
:205A8A00C0010000040F07430000050F4C0F02003E0610A102003E01130F02002006E0010C
:205AAA000000040F08430000050F4C0F02003E0610A102003E01180F020020060002000086
:205ACA00040F09430000050F4C0F02003E0610A102003E011D0F0200200620020000040F2D
:205AEA000A430000050F4C0F02003E0610A102003E01220F0200200640020000040F0B43AC
:205B0A000000050F4C0F02003E0610A102003E01270F0200200660020000040F0C430000B2
:205B2A00050F4C0F02003E0610A102003E012C0F0200200680020000040F0D430000050F58
:205B4A004C0F02003E0610A102003E01310F02002006A0020000040F0E430000050F4C0FCB
:205B6A0002003E0610A102003E01360F02002006C0020000040F0F430000050F4C0F0200DE
:205B8A003E0610A102003E013B0F02002006E0020000040F10430000050F4C0F02003E0656
:205BAA0010A102003E01400F0200200600030000040F11430000050F4C0F02003E0610A1A2
:205BCA0002003E01450F0200200620030000040F12430000050F4C0F02003E0610A102000B
:205BEA003E014A0F0200200640030000040F13430000050F4C0F02003E0660030000040F04
:205C0A0014430000050F00A302003E0100160200BE060E9E0200140F01000000240F00004A
:205C2A0000000C0F010070000411000000B48F700F0000001E0E000000003E5900007000C4
:205C4A000011000070000C11000000003E59000070000011000070000C11000000003E5960
:205C6A00000070000011000070000C11000000003E59000070000011000070000C11000067
:205C8A0000003E59000070000011000070000C110100700005110000700008113A8C02007D
:205CAA00140F000000923F7000000000340F000000203F0400000000240F000000003E5906
:205CCA0000000100010F010004003E01FFFF0000010F120204003E01021004003E010000AB
:205CEA0000803E5900100000010F00420000000F01007000001100007000011100420000CC
:205D0A00000F010070000011000070000110101102003E01750F0200200601000000010F48
:205D2A00328C0200011100430000000F010070000011000070000111D81502003E060000FE
:205D4A000000340F00160200BE0601430000010F010070000111000070000811000070004A
:205D6A00081100007000081100007000081100007000081100007000081100007000081153
:205D8A0000007000081100007000081100007000081100007000081100007000081100004C
:205DAA007000081100007000081100007000081100007000081100007000081100007000BC
:205DCA00081100007000081100007000081101000000240F000000000C0F00010000040F2B
:205DEA00EC150200BE0620010000040FEC150200BE0640010000040FEC150200BE0660015B
:205E0A000000040FEC150200BE0680010000040FEC150200BE06A0010000040FEC1502008C
:205E2A00BE06C0010000040FEC150200BE06E0010000040FEC150200BE0600020000040F29
:205E4A00EC150200BE0620020000040FEC150200BE0640020000040FEC150200BE066002F7
:205E6A000000040FEC150200BE0680020000040FEC150200BE06A0020000040FEC1502002A
:205E8A00BE06C0020000040FEC150200BE06E0020000040FEC150200BE0600030000040FC6
:205EAA00EC150200BE0620030000040FEC150200BE0640030000040FEC150200BE06600394
:205ECA000000040FEC150200BE063A8C0200140F00000000340F01000000240F000000007C
:205EEA00250FFFFF0000010F120204003E0100000100010F14000000680F040000001E0E33
:205F0A00000000007E59010004003E01021004003E01000000803E5900100000010F00428E
:205F2A000000000F01007000001100007000011100420000000F0100700000110000700001
:205F4A000110101102003E01D30F0200200601000000010F328C0200011100430000000F85
:205F6A00010070000011000070000111D81502003E06478D02000010488D02000210001100
:205F8A0002003E0168100200000610A102003E01E70F0200200680030000040F1543000038
:205FAA00050F341002003E0610A102003E01EC0F02002006A0030000040F16430000050F01
:205FCA00341002003E0610A102003E01F10F02002006C0030000040F17430000050F34108B
:205FEA0002003E0610A102003E01F60F02002006E0030000040F18430000050F3410020087
:20600A003E0610A102003E01FB0F0200200600040000040F19430000050F341002003E06FD
:20602A0010A102003E0100100200200620040000040F1A430000050F341002003E0610A149
:20604A0002003E0105100200200640040000040F1B430000050F341002003E0610A10200B2
:20606A003E010A100200200660040000040F1C430000050F341002003E0610A102003E012F
:20608A000F100200200680040000040F1D430000050F341002003E0610A102003E01141004
:2060AA0002002006A0040000040F1E430000050F341002003E0610A102003E0119100200DB
:2060CA002006C0040000040F1F430000050F341002003E0610A102003E011E100200200671
:2060EA00E0040000040F20430000050F341002003E0610A102003E0123100200200600054C
:20610A000000040F21430000050F341002003E0610A102003E0128100200200620050000E9
:20612A00040F22430000050F341002003E0610A102003E012D100200200640050000040F90
:20614A0023430000050F341002003E0610A102003E0132100200200660050000040F2443F6
:20616A000000050F341002003E0680050000040F25430000050F00A302003E01010070000E
:20618A00041100160200BE060E9E0200140F01000000240F000000000C0F000000B48F7031
:2061AA000F0000001E0E000000003E59000070000011000070000C11000000003E5900005E
:2061CA0070000011000070000C11000000003E59000070000011000070000C110000000002
:2061EA003E59000070000011000070000C11000000003E59000070000011000070000C114B
:20620A000100700005110000700008114E8C0200140F000000923F7000000000340F0000E1
:20622A0000203F0400000000240F000000003E5900000100010F010004003E01FFFF0000D4
:20624A00010F120204003E01021004003E01000000803E5900100000010F00420000000FF0
:20626A0001007000001100007000011100420000000F01007000001100007000011010119B
:20628A0002003E015D100200200601000000010F328C0200011100430000000F0100700078
:2062AA000011000070000111D81502003E0600000000340F00160200BE0615430000010F87
:2062CA0001007000011100007000081100007000081100007000081100007000081100000D
:2062EA00700008110000700008110000700008110000700008110000700008110000700077
:20630A000811000070000811000070000811000070000811000070000811000070000811AD
:20632A0000007000081100007000081101000000240F000000000C0F80030000040FEC155B
:20634A000200BE06A0030000040FEC150200BE06C0030000040FEC150200BE06E003000070
:20636A00040FEC150200BE0600040000040FEC150200BE0620040000040FEC150200BE065D
:20638A0040040000040FEC150200BE0660040000040FEC150200BE0680040000040FEC15FF
:2063AA000200BE06A0040000040FEC150200BE06C0040000040FEC150200BE06E00400000D
:2063CA00040FEC150200BE0600050000040FEC150200BE0620050000040FEC150200BE06FB
:2063EA0040050000040FEC150200BE0660050000040FEC150200BE0680050000040FEC159C
:20640A000200BE064E8C0200140F00000000340F01000000240F00000000250FFFFF000004
:20642A00010F120204003E0100000100010F11000000680F040000001E0E000000007E594B
:20644A00010004003E01021004003E01000000803E5900100000010F00420000000F010010
:20646A007000001100007000011100420000000F0100700000110000700001101011020098
:20648A003E01B2100200200601000000010F328C0200011100430000000F01007000001112
:2064AA00000070000111D81502003E0646534821020F212200003E01C6100200200600107A
:2064CA000000010F00420000000F010070000011000070000111F9090200BE06D815020096
:2064EA003E0646535421020F212200003E01F21002002006468D02000110101102003E013B
:20650A00DF1002002006478D02000110488D0200021010A102003E01000000921F700A422B
:20652A000000000F011100003E010100700001110000700002113A8C0200140F0000000000
:20654A00340F000000203F0400000000240F000000003E59FFFF0000010F010004003E016F
:20656A00221000003E02021004003E01000000803E59D81502003E06478D02000110488D44
:20658A000200021010A102003E01000000921F701E420000000F011100003E010100700099
:2065AA0001110000700002114E8C0200140F00000000340F000000203F0400000000240F64
:2065CA00000000003E59FFFF0000010F010004003E01221000003E02021004003E01000001
:2065EA0000803E59D81502003E0646545021020F212200003E01FC1002002006468D0200A0
:20660A000110101102003E01FA1002000006040000000014FB1002003E060400000020144A
:20662A00D81502003E0647454E21020F212200003E010A1102002006468D020001108B8C4F
:20664A0002000111478D020001108C8C02000111488D020001108D8C02000111498D02001C
:20666A0001108A8C020001114A8D02000110918C02000111D81502003E0649445021020F78
:20668A00212200003E012D1102002006468D0200011070A102000111478D0200011071A104
:2066AA0002000111488D0200011073A102000111498D02000110ECA1020001114A8D020049
:2066CA000110EDA1020001114B8D02000110101102003E011C11020000060800000000145F
:2066EA001D1102003E060800000020144C8D02000110101102003E01221102000006100047
:20670A0000000014231102003E0610000000201470A1020000107BA1020001100122000028
:20672A003E017FEE0200021120A202003E017EEE0200021171A10200001000A002003E0105
:20674A0080EE02000011D81502003E064C454421020F212200003E01331102002006468DB3
:20676A0002000110868C02000111D81502003E064D445421020F212200003E013E110200B9
:20678A002006328C0200011001000000020F122104003E0100430000000F0100700000119C
:2067AA00000070000111328C02000111D81502003E064E434621020F212200003E01541158
:2067CA0002002006468D0200150F00000000350F01000000240F00000000250F0000800062
:2067EA003E5B76A1020001114FEC02000111A7A10200140F00000000340F10000000680F45
:20680A00020000001E0E000080003E5B000080803E59B7A10200140F10000000680F02008A
:20682A0000001E0E000080003E5B000080803E59D81502003E064E434E21020F21220000EB
:20684A003E0102120200200600000000010F328C02000111468D020001106CA102000111CA
:20686A0010A102003E01641102002406FEFFFFFF030F00040000000FFEFFFFFF040FFFFF4F
:20688A00FFFF050FE91102043E06F00A0000010FF00A0000020F10A102003E016D11020011
:2068AA002406FCFFFFFF030F00020000000FFEFFFFFF040FFDFFFFFF050FE91102043E0628
:2068CA0078050000010F78050000020F10A102003E01761102002406F8FFFFFF030F540192
:2068EA000000000FFAFFFFFF040FFDFFFFFF050FE91102043E06A5030000010FA5030000C3
:20690A00020F10A102003E017F110200240600010000000FF0FFFFFF030FFAFFFFFF040F95
:20692A00F5FFFFFF050FE91102043E06BC020000010FBC020000020F10A102003E018811DB
:20694A0002002406E0FFFFFF030FC8000000000FEAFFFFFF040FF5FFFFFF050FE91102043B
:20696A003E0630020000010F30020000020F10A102003E01911102002406C0FFFFFF030FB5
:20698A00AA000000000FEAFFFFFF040FD5FFFFFF050FE91102043E06D1010000010FD1015C
:2069AA000000020F10A102003E019A110200240680FFFFFF030F91000000000FAAFFFFFF1D
:2069CA00040FD5FFFFFF050FE91102043E0690010000010F90010000020F10A102003E013B
:2069EA00A3110200240680000000000F00FFFFFF030FAAFFFFFF040F55FFFFFF050FE911F5
:206A0A0002043E065E010000010F5E010000020F10A102003E01AC110200240600FEFFFF6C
:206A2A00030F71000000000FAAFEFFFF040F55FFFFFF050FE91102043E0637010000010F0F
:206A4A0037010000020F10A102003E01B5110200240600FCFFFF030F66000000000FAAFED6
:206A6A00FFFF040F55FDFFFF050FE91102043E0618010000010F18010000020F10A102004D
:206A8A003E01BE11020024065D000000000F00F8FFFF030FAAFAFFFF040F55FDFFFF050F25
:206AAA00E91102043E06FE000000010FFE000000020F10A102003E01C7110200240600F085
:206ACA00FFFF030F55000000000FAAFAFFFF040F55F5FFFF050FE91102043E06E9000000FA
:206AEA00010FE9000000020F10A102003E01D0110200240600E0FFFF030F4E000000000F36
:206B0A00AAEAFFFF040F55F5FFFF050FE91102043E06D7000000010FD7000000020F10A1A6
:206B2A0002003E01D9110200240600C0FFFF030F49000000000FAAEAFFFF040F55D5FFFFFF
:206B4A00050FE91102043E06C8000000010FC8000000020F10A102003E01E2110200240611
:206B6A0044000000000F0080FFFF030FAAAAFFFF040F55D5FFFF050FE91102043E06BA0089
:206B8A000000010FBA000000020F40000000000F0000FFFF030FAAAAFFFF040F5555FFFFA4
:206BAA00050FE91102043E06AF000000010FAF000000020FC7A102000111CBA102000011F9
:206BCA00CAA102000011C8A10200021100000000000F001002003E01FB110200000601003A
:206BEA000000000F001002003E01F7110200000676A102000010041004003E0176A1020082
:206C0A000011FE1102003E0676A102000010051004003E0176A102000011FE1102003E0604
:206C2A0076A102000010031004003E0176A102000011F9090200BE0601000000010F328C0A
:206C4A0002000111D81502003E064E455221020F212200003E010D12020020060000000003
:206C6A00010F328C02000111468D020001106DA102000111F9090200BE0601000000010F47
:206C8A00328C02000111D81502003E064E524621020F212200003E012912020020060000E8
:206CAA000000010F328C02000111468D020001106BA10200011110A102003E0119120200C3
:206CCA002006251202043E06F00A0000010FC9A10200011110A102003E011E120200200631
:206CEA00251202043E0678050000010FC9A10200011110A102003E01231202002006251278
:206D0A0002043E06A5030000010FC9A102000111BC020000010FC9A102000111F909020099
:206D2A00BE0601000000010F328C02000111D81502003E064F52533F020F212200003E01A9
:206D4A003B12020020060B000000000F659502000011C6ED0200140F00000000340F04006E
:206D6A000000240F64950200110F00000000310F000000603E0401000000240F1400000091
:206D8A00680F020000001E0E000080003E59000080803E53D1150200BE06C21502003E06D3
:206DAA005244593F020F212200003E014A1202002006D1150200BE0652445921010F6895BB
:206DCA000200011111F000783E026995020001110A000000010F6A9502000111000000009D
:206DEA00010F6B950200011103000000000F659502000011C21502003E0652454621020F1A
:206E0A00212200003E018A120200200600000000000F328C020000117EA10200100F000002
:206E2A000000300F7FA10200001180A10200001181A10200001182A1020000110100000036
:206E4A00010F468D0200211097A102002111000080807E40478D0200211098A10200211174
:206E6A00000080807E40488D0200211099A102002111000080807E40498D020021109AA1D2
:206E8A0002002111000080807E404A8D020021109BA102002111000080807E404B8D0200E4
:206EAA0021109CA102002111000080807E404C8D020021109DA102002111000080807E402C
:206ECA004D8D020021109EA102002111000080807E404E8D020021109FA1020021110000E8
:206EEA0080807E404F8D02002110A0A102002111000080807E40508D02002110A1A1020034
:206F0A002111000080807E40518D02002110A2A102002111000080807E40528D020021101F
:206F2A00A3A102002111000080807E40538D02002110A4A102002111000080807E40548DE6
:206F4A0002002110A5A102002111000080807E40558D02002110A6A102002111000080802C
:206F6A007E40F9090200BE0601000000010F328C02000111D81502003E06524E5021020F49
:206F8A00212200003E01901202002006468D02000110BA8C02000111D81502003E06525383
:206FAA005421020F212200003E01B0120200200600000000010F328C0200011100430000B0
:206FCA00000F01007000001100007000011100420000000F01007000001100100000010FA1
:206FEA00000070000111468D02000110101102003E01A0120200200666EC02000111478DA9
:20700A0002000110101102003E01A4120200200667EC02000111F9090200BE0600420000A2
:20702A00000F010070000011000070000110101102003E01A5120200200601000000010FE2
:20704A00328C0200011100430000000F010070000011000070000111D81502003E06534137
:20706A004D21020F212200003E01731302002006468D02000110478D02000210488D0200B2
:20708A00031000430000000F01007000001100000000000F000070000011328C020000119E
:2070AA0089150000000F012400003E01C81202002006878C0200001151C80000000F004421
:2070CA00AC45010F201202003E013D130200000600442C44010F301302003E013D13020040
:2070EA000006FE43AC42010F3D1302003E06D7190000000F012400003E01D5120200200639
:20710A00878C020000115FC80000000F00B8CE45010F201202003E013D130200000600B8AB
:20712A004E44010F301302003E013D130200000603B8CE42010F3D1302003E06401F0000F7
:20714A00000F012400003E01E21202002006878C0200001150C80000000F0000FA45010FFA
:20716A00201202003E013D130200000600007A44010F301302003E013D1302000006000090
:20718A00FA42010F3D1302003E0680250000000F012400003E01EF1202002006878C0200AD
:2071AA0000115EC80000000F00001646010F201202003E013D130200000600009644010F5E
:2071CA00301302003E013D130200000600001643010F3D1302003E06112B0000000F01245A
:2071EA0000003E01FC1202002006878C0200001153C80000000F00442C46010F20120200C6
:20720A003E013D13020000060044AC44010F301302003E013D1302000006FE432C43010FED
:20722A003D1302003E06803E0000000F012400003E01091302002006878C0200001152C8F9
:20724A000000000F00007A46010F201202003E013D13020000060000FA44010F30130200E7
:20726A003E013D130200000600007A43010F3D1302003E06D4490000000F012400003E017A
:20728A00161302002006878C0200001155C80000000F00A89346010F201202003E013D13ED
:2072AA000200000600A81345010F301302003E013D130200000600A89343010F3D130200F0
:2072CA003E0622560000000F012400003E01231302002006878C0200001157C80000000FC3
:2072EA000044AC46010F201202003E013D130200000600442C45010F301302003E013D13DA
:20730A0002000006F843AC43010F3D1302003E06256B0000000F012400003E013013020043
:20732A002006878C0200001154C80000000F2449D646010F201202003E013D130200000668
:20734A001F495645010F301302003E013D13020000061749D643010F3D1302003E06007D98
:20736A000000000F012400003E01BE1202002006878C0200001156C80000000F0000FA4605
:20738A00010F201202003E013D130200000600007A45010F301302003E013D13020000065D
:2073AA0000409C45010F3D1302003E06BB8C02000111A6050200BE06B6050200BE06B605F4
:2073CA000200BE06FF0F0000040F040004003E01A6050200BE06C8000000680F02000000C3
:2073EA001E0EB6050200BE0600000000000001420000000F0100700000110000700002117F
:20740A0002420000000F010070000011000070000311888C02000211898C020003111E0097
:20742A000000040F201202003E0157130200000605000000040F301302003E015713020042
:20744A00000602000000040F7BA10200041170A1020000107BA102000110012200003E0120
:20746A007FEE0200021120A202003E017EEE0200021171A10200001000A002003E0180EE89
:20748A0002000011B6050200BE0651070200BE06F9090200BE0600100000010F0042000006
:2074AA00000F01007000001100007000011100420000000F0100700000110000700001105B
:2074CA00101102003E0168130200200601000000010F328C0200011100430000000F010067
:2074EA0070000011000070000111D81502003E0653444521020F212200003E01A113020006
:20750A00200661E80200110F00000000310F01000000200FAC030000680F010000001E0E0D
:20752A0000000000009200000000080F0A000000090F468D0200100F00000000300F61E8FA
:20754A000200110F00000000000F01000000010F000080811F71000000403E0417000000B5
:20756A00680F070000001E0E000000013E50201202003E018D1302000006000080803E521D
:20758A00000000813E52009002003E01109102003E01000080801F71000080883F700000D6
:2075AA0000803E52000080881F70809802003E01982000003E01811302002406000000000A
:2075CA00000F328C0200001161E80200110FF9E30200100FAC030000680F020000001E0E05
:2075EA00000000003E52000000803E50F9090200BE0601000000000F328C02000011D8154D
:20760A0002003E065344453F020F212200003E01CF1302002006D1150200BE06CC010000E9
:20762A00000F009002003E0165950200001161E80200110F00000000310F01000000200F78
:20764A00AC030000680F010000001E0E00000000009200000000080F0A000000090FF9E326
:20766A000200100F00000000300F61E80200110F17000000210F000000003E50001002004E
:20768A003E01C01302000006000000821F7107000000000D000000003E5000A002003E0131
:2076AA00000000910F70000000003E50000080884F70000000503E04000000803E520000B9
:2076CA0080884F70000000483E04809802003E01982000003E01B41302002406689502000D
:2076EA00100F00000000300F61E80200110FCC010000010F04000000010D000080003E52B8
:20770A00000080803E5011F000783E02000080803E50C21502003E0653445221020F21220F
:20772A0000003E01FD130200200661E80200110F00000000310F01000000200FBC00000031
:20774A00680F010000001E0E00000000009200000000080F04000000090F468D0200100FC2
:20776A0000000000300F61E80200110F00000000000F01000000010F000080811F710000A4
:20778A0000403E0417000000680F070000001E0E000000013E50201202003E01E91302009C
:2077AA000006000080803E52000000813E52009002003E01109102003E01000080801F71D5
:2077CA00000080883F70000000803E52000080881F70809802003E01982000003E01DD1301
:2077EA000200240600000000000F328C0200001161E80200110FA5E70200100FBC0000009F
:20780A00680F020000001E0E000000003E52000000803E50F9090200BE0601000000000F43
:20782A00328C02000011D81502003E065344523F020F212200003E012B1402002006D11532
:20784A000200BE06CC010000000F009002003E0165950200001161E80200110F0000000033
:20786A00310F01000000200FBC000000680F010000001E0E00000000009200000000080F85
:20788A0004000000090FA5E70200100F00000000300F61E80200110F17000000210F000024
:2078AA0000003E50001002003E011C1402000006000000821F7107000000000D0000000081
:2078CA003E5000A002003E01000000910F70000000003E50000080884F70000000503E0438
:2078EA00000000803E52000080884F70000000483E04809802003E01982000003E011014A9
:20790A000200240668950200100F00000000300F61E80200110FCC010000010F0400000088
:20792A00010D000080003E52000080803E5011F000783E02000080803E50C21502003E062D
:20794A005349443F020F212200003E013E1402002006D1150200BE064E4F5641010F689504
:20796A000200011111F000783E0269950200011143533220010F6A950200011111F000789A
:20798A003E026B950200011153445320010F6C950200011111F000783E026D95020001118B
:2079AA0004000000000F659502000011C21502003E0653465121020F212200003E01551479
:2079CA0002002006468D020001108E8C02000111478D020001108F8C02000111488D020074
:2079EA000110908C02000111498D02000110B48C020001114A8D02000110B58C02000111C0
:207A0A004B8D02000110B68C020001110A8D0200011084EE0200011100000000010F0A8D44
:207A2A000200011151070200BE0684EE020001100A8D02000111D81502003E06534D502196
:207A4A00020F212200003E0169140200200677BE7F3F030F468D02000110312408003E015D
:207A6A005D140200220677BE7F3F010FB78C02000111478D02000110312408003E0162140E
:207A8A000200220677BE7F3F010FB88C02000111488D02000110312408003E016714020056
:207AAA00220677BE7F3F010FB98C02000111D81502003E0653524321020F212200003E0169
:207ACA00741402002006468D020001100A000000000F012000003E0172140200200651EEA0
:207AEA000200001153EE02000011928C02000111D81502003E065354533F020F2122000023
:207B0A003E01C21402002006D1150200BE0675A10200011068950200011111F000783E027F
:207B2A0069950200011174A1020001106A950200011111F000783E026B9502000111000021
:207B4A000000010F75A10200011174A1020001114FEE020001106C950200011111F00078DA
:207B6A003E026D950200011100000000010F4FEE020001110000200080148C1402003A06AE
:207B8A0001000000010F6E950200011111F000783E026F95020001110000200020144FEC53
:207BAA000200011070950200011111F000783E0271950200011100000000010F00000001AB
:207BCA008014981402003A0601000000010F72950200011111F000783E0273950200011118
:207BEA0000000001201468EE0200011074950200011111F000783E027595020001110000E9
:207C0A000000010F68EE020001117AA10200011076950200011111F000783E0277950200CC
:207C2A00011100000000010F7AA102000111000000048014AB1402003A0601000000010F3F
:207C4A0078950200011111F000783E02799502000111000000042014AA8C020001107A958E
:207C6A000200011111F000783E027B9502000111AB8C020001107C950200011111F0007821
:207C8A003E027D9502000111AF8C020001107E950200011111F000783E027F95020001111E
:207CAA00B08C0200011080950200011111F000783E028195020001110E000000000F659548
:207CCA0002000011C21502003E0654504221020F212200003E012015020020060000000073
:207CEA00020F468D02000110B7A102000111212100003E011E1502008206478D02000110F2
:207D0A00B8A102000111212100003E011E1502008206488D02000110B9A102000111212116
:207D2A0000003E011E1502008206498D02000110BAA102000111212100003E011E1502002F
:207D4A0082064A8D02000110BBA102000111212100003E011E15020082064B8D020001100E
:207D6A00BCA102000111212100003E011E15020082064C8D02000110BDA1020001112121AA
:207D8A0000003E011E15020082064D8D02000110BEA102000111212100003E011E150200C7
:207DAA0082064E8D02000110BFA102000111212100003E011E15020082064F8D02000110A2
:207DCA00C0A102000111212100003E011E1502008206508D02000110C1A10200011121213E
:207DEA0000003E011E1502008206518D02000110C2A102000111212100003E011E1502005F
:207E0A008206528D02000110C3A102000111212100003E011E1502008206538D0200011035
:207E2A00C4A102000111212100003E011E1502008206548D02000110C5A1020001112121D1
:207E4A0000003E011E1502008206558D02000110C6A102000111212100003E011E150200F6
:207E6A00820679A102000211003402001C0F000000003C0F003402001D0F000000003D0FE7
:207E8A00010000002C0FCBA102002D1000000081DF7200000000030FB7A10200140F000090
:207EAA000000340F01000000240F6CA102006810090000001E0E000080003E5900000097D7
:207ECA001F70000000307F04212100003E0101000000010D000080813F59000000687F0442
:207EEA0000008080DF710000008E1F70D81502003E06000000811F70000000003E0A5450DC
:207F0A004621020F212200003E017C150200200600000000020F468D02000110A7A1020063
:207F2A000111212100003E011E1502008206478D02000110A8A102000111212100003E0122
:207F4A001E1502008206488D02000110A9A102000111212100003E011E1502008206498D00
:207F6A0002000110AAA102000111212100003E011E15020082064A8D02000110ABA102000F
:207F8A000111212100003E011E15020082064B8D02000110ACA102000111212100003E01BA
:207FAA001E15020082064C8D02000110ADA102000111212100003E011E15020082064D8D94
:207FCA0002000110AEA102000111212100003E011E15020082064E8D02000110AFA10200A3
:207FEA000111212100003E011E15020082064F8D02000110B0A102000111212100003E0152
:20800A001E1502008206508D02000110B1A102000111212100003E011E1502008206518D27
:20802A0002000110B2A102000111212100003E011E1502008206528D02000110B3A1020036
:20804A000111212100003E011E1502008206538D02000110B4A102000111212100003E01E9
:20806A001E1502008206548D02000110B5A102000111212100003E011E1502008206558DBB
:20808A0002000110B6A102000111212100003E011E150200820678A10200021100300200BA
:2080AA001C0F000000003C0F003002001D0F000000003D0F010000002C0FCBA102002D10AF
:2080CA0000000081DF7200000000030FA7A10200140F00000000340F01000000240F6CA1C1
:2080EA0002006810090000001E0E000080003E59000000971F70000000307F042121000095
:20810A003E0101000000010D000080813F59000000687F0400008080DF710000008E1F7016
:20812A00D81502003E0655535421020F212200003E01861502002006468D020001100000A9
:20814A0000810F770000FFFF030F230204003E01121204003E01000000B82F70D8150200E9
:20816A003E0657475421020F212200003E01C21502002006468D02000010478D0200011040
:20818A00488D02000210498D020003104A8D0200041000A002003E01A7150200000600006F
:2081AA000000050F00004200180F00000000380F01000000280FCAA102002D10800000008F
:2081CA002F0F509502003E01452700003E01A115020000066CA102006810010000001E0E14
:2081EA00000000287E04000000387E04000000387E04000000387E04000000387E04961538
:20820A0002003E0630A302003E01B31502000006000000B43F70010000001E0E0000002872
:20822A007E04B31502003E06101102003E0100300200180FAD150204000600000000380FD4
:20824A0001000000280F00340200180F30A302003E01B31502000006CBA1020029100000F4
:20826A0000B43F70010000001E0E000000087E04000000B42F70209402003E016595020096
:20828A00041104000000240F64950200110F00000000310F000000603E0401000000210F5A
:2082AA00040000001E0E000080003F50000080807E5211F000783E02000080807E52D11536
:2082CA000200BE06C21502003E0664950200000F78000000001101000000000F7900000095
:2082EA00001120080000000F7A000000001100000000030FF0000000031100000000000F7C
:20830A00899D02000011859D02000310F00000000311000000043E0A00000000000F849D63
:20832A000200001101000000000F64950200001143310000010F669502000111000000046D
:20834A003E0A50430000010F679502000111D1150200BE068CEE02000110689502000111CE
:20836A0011F000783E02699502000111204F4B0A010F6A950200011111F000783E026B9588
:20838A000200011103000000000F659502000011C21502003E0668950200011111F00078F9
:2083AA003E02699502000111D1150200BE0602000000000F659502000011C21502003E067A
:2083CA00E41502003E060100700004110E9E0200140F000000B48F700F0000001E0E00000F
:2083EA0000003E59000070000011000070000C11000000003E590000700000110000700046
:20840A000C11000000003E59000070000011000070000C11000000003E5900007000001178
:20842A00000070000C11000000003E59000070000011000070000C11000000003E0AFF00B9
:20844A0000000C0F2C0C04003E01CE9D0200140F00000092CF70000000203F0400000004B4
:20846A003E598E9D0200140F000000203F04000000003E590000008A0F7001000000240FD4
:20848A000E9E0200100F00000000300F000000B48F700A0000001E0E000000003E59000046
:2084AA0000803E51000000003E59000000803E51000000003E59000000803E510000000057
:2084CA003E59000000803E51000000003E59000000803E5100FF00000C0F2C0C04003E01B1
:2084EA00CCF800783E02CE9D0200140F00000092CF70000000203F04000000063E598C18F1
:20850A0000003E018E9D0200140F000000203F04000000003E590000008A0F7001000000BE
:20852A00240F000000B4CF700A0000001E0E000000003E59000000803E51000000003E5998
:20854A00000000803E51000000003E59000000803E51000000003E59000000803E510000B6
:20856A0000003E59000000803E51000000003E0A6CA102000410402400003E01000000003D
:20858A00020A00300200180F00000000380F01000000280FCBA10200291000A402003E0161
:2085AA003F1602000006000000B44F70010000001E0E000000087E0400000000040F000017
:2085CA0000B49F72010000001E0E000000823F5000340200180F00A402003E0149160200EB
:2085EA000006000000B44F70010000001E0E000000087E0400000000040F000000B49F7269
:20860A00010000001E0E000000823F50F00A0000340F23AD0200440F13B8020014100100BE
:20862A000000240FC7A10200251000A402003E01571602000006000000B44F700100000090
:20864A001E0E000000283F04000000B49F72010000001E0E000000000099000000003E0AA6
:20866A00000007000A14008000002A14000070002C14D5070200BE0601000000000F8041EA
:20868A000000010F010070000111000070000110012100003E016016020020066620000037
:2086AA00000F00420000010F010070000111000070000011FC040200BE0601000000000F75
:2086CA00001002003E016E1602000006791D0200BE0601000000010F328C02000111004331
:2086EA000000000F010070000011000070000111928C020001100A000000000F01200000F2
:20870A003E017C1602000006C1050200BE06849D02000010001002003E01230B0200A00690
:20872A00731602003E06010000008014A91602003A068EEE020070110000100000140000A7
:20874A000800201402000000201400000000000F8FEE02000011C1050200BE06849D02004F
:20876A000010001002003E01230B0200A006000002000014000002008014891602001A064B
:20878A0057040200BE067E1A0200BE068FEE02000010009002003E018FEE02000011C80098
:2087AA000000010F012000003E01841602002006000010002014000008000014000000001D
:2087CA00000F8FEE02000011C1050200BE06849D02000010001002003E01230B0200A0060A
:2087EA000000020000140000020080149C1602001A0657040200BE067E1A0200BE068FEEF3
:20880A0002000010009002003E018FEE02000011C8000000010F012000003E0197160200F4
:20882A0020068EEE02007010000008000014000010000014C1050200BE06849D020000100B
:20884A00001002003E01230B0200A006928C020001100A000000000F012000003E01A9167E
:20886A0002002006010000008014E11602003A06C5ED02000010009002003E01C5ED0200AF
:20888A00001173A102000110102100003E01E1160200240600000000020FC5ED020002112B
:2088AA00020000008014D71602003A06C4ED02000010009002003E01C4ED0200001172A17E
:2088CA0002000110102100003E01D71602002406C4ED02000211000006000014000006000C
:2088EA008014C51602001A0657040200BE0695040200BE067E1A0200BE064EEC02000010B3
:20890A0074A10200001100000000000F4EEC02000011849D02000010001002003E01230B17
:20892A000200A006F31B0200BE064DEC0200001075A10200001100000000000F4DEC0200F3
:20894A000011A91602003E06000002000014000002008014D81602001A0657040200BE061A
:20896A007E1A0200BE064EEC0200001074A10200001100000000000F4EEC02000011A91600
:20898A0002003E06020000008014F51602003A06C4ED02000010009002003E01C4ED02005D
:2089AA00001172A102000110102100003E01F5160200240600000000020FC4ED02000211F8
:2089CA00000004000014000004008014EC1602001A0695040200BE06F31B0200BE064DEC4D
:2089EA000200001075A10200001100000000000F4DEC02000011A91602003E0600000100D1
:208A0A000014000001008014F61602001A06A91602003E0691EE0200140F00000000340F89
:208A2A000000803F070F00088B087E6800100A828F7070270A000201410413003E0140912F
:208A4A000C003E01010033003E0270270A00300110A40C003E01000080087E68140C930853
:208A6A007E68401C59003E01C128080A7E68800C0B003E01C42408868F70121702000206B3
:208A8A00CC0C130A7E6802000006000CC40493087E68141408003E01C40413003E014804BF
:208AAA0013043E0A481C08003E01C70013003E01000000003E0AAA8C020000109EEE02006B
:208ACA000011AB8C020000109FEE02000011AF8C02000010A0EE02000011B08C0200001056
:208AEA00A1EE02000011C48C0200100F00000000300F348C0200110F00000000310F0100F7
:208B0A000000210F80000000680F020000001E0E000000007E50000000807E5277A10200BE
:208B2A000010000000B80F7000001000001400000800001470A1020000107BA10200011052
:208B4A00012200003E017FEE0200021120A202003E017EEE0200021171A10200001000A0DF
:208B6A0002003E0180EE02000011EAA10200001070EC0200100FA0000000680F01000000F7
:208B8A001E0E000000803E50EAA1020000100000803E010F010013003E0110ED0200100FB5
:208BAA00A0000000680F010000001E0E000000803E50EAA102000010EBA10200011001001C
:208BCA0013003E010000803F010F102108003E0150EC02000111DAED0200100F00000000BA
:208BEA00300F01000000200F14000000680F010000001E0E000080803E500B100000000F8C
:208C0A00358C0200001104000000000FAC8C0200001109000000000FAD8C020000110A00AA
:208C2A000000000FAE8C020000110A000000000F368C0200001109000000000F378C020003
:208C4A00001167000000000FB38C0200001101000000000FA98C020000119EEE020000103B
:208C6A00AA8C020000119FEE02000010AB8C02000011A0EE02000010AF8C02000011A1EE3B
:208C8A0002000010B08C0200001100000080AF77000000C0010F010104003E0111E2007843
:208CAA003E02B18C0200011100000030010F010104003E0111E400783E02B28C0200011195
:208CCA00A7A10200100F00000000300F01000000200F00000000000F10000000680F050017
:208CEA0000001E0E000080003E50102200003E01751702000406000000801F700000000018
:208D0A00000078A102000011B7A10200100F00000000000F10000000680F050000001E0EDD
:208D2A00000080003E50102200003E017F1702000406000000801F7000000000000079A1DF
:208D4A000200001197A10200100F01000000010F10000000680F0F0000001E0E00000000CA
:208D6A003E5000A002003E018A17020020067FA102000111931702003E0600A002003E01AC
:208D8A008E170200200680A102000111931702003E0600A002003E0192170200200681A103
:208DAA0002000111931702003E0682A10200011100000000000000002000201400004000DA
:208DCA00201400008000201400000001201400000002201400000004201400000000000FEF
:208DEA004DEC020000114EEC02000011C4ED02000011C5ED0200001116EE020000114FEEF3
:208E0A000200001118EE0200001168EE0200001174A10200001175A10200001151EE020021
:208E2A00001153EE020000116DEC0200001117EE0200001176A1020001104FEC02000111C6
:208E4A006CA10200011010A102003E01B51702002406FEFFFFFF030F00040000000FFEFFE1
:208E6A00FFFF040FFFFFFFFF050F3A1802043E06F00A0000010FF00A0000020F10A1020063
:208E8A003E01BE1702002406FCFFFFFF030F00020000000FFEFFFFFF040FFDFFFFFF050F50
:208EAA003A1802043E0678050000010F78050000020F10A102003E01C71702002406F8FFFE
:208ECA00FFFF030F54010000000FFAFFFFFF040FFDFFFFFF050F3A1802043E06A5030000B8
:208EEA00010FA5030000020F10A102003E01D0170200240600010000000FF0FFFFFF030F8B
:208F0A00FAFFFFFF040FF5FFFFFF050F3A1802043E06BC020000010FBC020000020F10A14D
:208F2A0002003E01D91702002406E0FFFFFF030FC8000000000FEAFFFFFF040FF5FFFFFF18
:208F4A00050F3A1802043E0630020000010F30020000020F10A102003E01E21702002406BB
:208F6A00C0FFFFFF030FAA000000000FEAFFFFFF040FD5FFFFFF050F3A1802043E06D10111
:208F8A000000010FD1010000020F10A102003E01EB170200240680FFFFFF030F9100000094
:208FAA00000FAAFFFFFF040FD5FFFFFF050F3A1802043E0690010000010F90010000020F19
:208FCA0010A102003E01F4170200240680000000000F00FFFFFF030FAAFFFFFF040F55FFB2
:208FEA00FFFF050F3A1802043E065E010000010F5E010000020F10A102003E01FD170200D2
:20900A00240600FEFFFF030F71000000000FAAFEFFFF040F55FFFFFF050F3A1802043E06D3
:20902A0037010000010F37010000020F10A102003E0106180200240600FCFFFF030F6600E7
:20904A000000000FAAFEFFFF040F55FDFFFF050F3A1802043E0618010000010F18010000FC
:20906A00020F10A102003E010F18020024065D000000000F00F8FFFF030FAAFAFFFF040F67
:20908A0055FDFFFF050F3A1802043E06FE000000010FFE000000020F10A102003E01181887
:2090AA000200240600F0FFFF030F55000000000FAAFAFFFF040F55F5FFFF050F3A180204AD
:2090CA003E06E9000000010FE9000000020F10A102003E0121180200240600E0FFFF030F08
:2090EA004E000000000FAAEAFFFF040F55F5FFFF050F3A1802043E06D7000000010FD700AE
:20910A000000020F10A102003E012A180200240600C0FFFF030F49000000000FAAEAFFFF1A
:20912A00040F55D5FFFF050F3A1802043E06C8000000010FC8000000020F10A102003E0197
:20914A0033180200240644000000000F0080FFFF030FAAAAFFFF040F55D5FFFF050F3A18B8
:20916A0002043E06BA000000010FBA000000020F40000000000F0000FFFF030FAAAAFFFF55
:20918A00040F5555FFFF050F3A1802043E06AF000000010FAF000000020FC7A1020001115F
:2091AA00CBA102000011CAA102000011C8A1020002116BA10200011010A102003E014418BD
:2091CA0002002006501802043E06F00A0000010FC9A10200011110A102003E0149180200CE
:2091EA002006501802043E0678050000010FC9A10200011110A102003E014E180200200602
:20920A00501802043E06A5030000010FC9A102000111BC020000010FC9A102000111000010
:20922A000000000F001002003E015E180200000601000000000F001002003E015A18020071
:20924A00000676A102000010041004003E0176A102000011611802003E0676A1020000106C
:20926A00051004003E0176A102000011611802003E0676A102000010031004003E0176A10D
:20928A0002000011F9090200BE06EF8C020003105F8C02000311F18C02000410618C0200D6
:2092AA000411F38C02000510638C02000511F58C02000610658C02000611F78C02000710B3
:2092CA00678C020007116E1A0200BE06B6050200BE06B6050200BE0600010000000FF08C9B
:2092EA0002000310031304003E01608C02000311F28C02000410041404003E01628C020015
:20930A000411F48C02000510051504003E01648C02000511F68C02000610061604003E0139
:20932A00668C02000611F88C02000710071704003E01688C020007116E1A0200BE06B60503
:20934A000200BE06B6050200BE0600060000000F038D02000310031304003E01738C0200A8
:20936A000311058D02000410041404003E01758C02000411078D02000510051504003E01AC
:20938A00778C02000511098D02000610061604003E01798C020006110B8D020007100717AE
:2093AA0004003E017B8C020007116E1A0200BE06B6050200BE06B6050200BE0600070000E8
:2093CA00000F048D02000310031304003E01748C02000311068D02000410041404003E015B
:2093EA00768C02000411088D02000510051504003E01788C020005110A8D0200061006165A
:20940A0004003E017A8C020006110C8D02000710071704003E017C8C020007116E1A020021
:20942A00BE06B6050200BE06B6050200BE06178D02000110878C02000111188D02000210C5
:20944A00888C02000211198D02000310898C0200031189150000000F012400003E01BB180F
:20946A0002002006878C0200001151C80000000F0044AC45010F201202003E013019020069
:20948A00000600442C44010F301302003E01301902000006FE43AC42010F301902003E0655
:2094AA00D7190000000F012400003E01C81802002006878C020000115FC80000000F00B823
:2094CA00CE45010F201202003E0130190200000600B84E44010F301302003E013019020072
:2094EA00000603B8CE42010F301902003E06401F0000000F012400003E01D518020020060B
:20950A00878C0200001150C80000000F0000FA45010F201202003E013019020000060000E1
:20952A007A44010F301302003E013019020000060000FA42010F301902003E0680250000FE
:20954A00000F012400003E01E21802002006878C020000115EC80000000F00001646010FA5
:20956A00201202003E0130190200000600009644010F301302003E0130190200000600005E
:20958A001643010F301902003E06112B0000000F012400003E01EF1802002006878C0200D6
:2095AA00001153C80000000F00442C46010F201202003E013019020000060044AC44010F98
:2095CA00301302003E01301902000006FE432C43010F301902003E06803E0000000F01246B
:2095EA0000003E01FC1802002006878C0200001152C80000000F00007A46010F2012020093
:20960A003E013019020000060000FA44010F301302003E0130190200000600007A43010FC0
:20962A00301902003E06D4490000000F012400003E01091902002006878C0200001155C874
:20964A000000000F00A89346010F201202003E0130190200000600A81345010F3013020047
:20966A003E0130190200000600A89343010F301902003E0622560000000F012400003E0148
:20968A00161902002006878C0200001157C80000000F0044AC46010F201202003E01301913
:2096AA000200000600442C45010F301302003E01301902000006F843AC43010F3019020079
:2096CA003E06256B0000000F012400003E01231902002006878C0200001154C80000000F84
:2096EA002449D646010F201202003E013019020000061F495645010F301302003E01301923
:20970A00020000061749D643010F301902003E06007D0000000F012400003E01B118020064
:20972A002006878C0200001156C80000000F0000FA46010F201202003E0130190200000692
:20974A0000007A45010F301302003E0130190200000600409C45010F301902003E06BB8C54
:20976A0002000111A6050200BE06B6050200BE06B6050200BE06FF0F0000040F040004002F
:20978A003E01A6050200BE06C8000000680F020000001E0EB6050200BE0600000000000021
:2097AA0001420000000F01007000001100007000021102420000000F010070000011000073
:2097CA0070000311888C02000211898C020003111E000000040F201202003E014A1902009E
:2097EA00000605000000040F301302003E014A190200000602000000040F7BA1020004110A
:20980A00B6050200BE0651070200BE06CA8C0200021001000000030F00010000040F0143CA
:20982A000000050F3A1A0200BE06CB8C0200021002000000030F20010000040F02430000F8
:20984A00050F3A1A0200BE06CC8C0200021003000000030F40010000040F03430000050FA1
:20986A003A1A0200BE06CD8C0200021004000000030F60010000040F04430000050F3A1A1E
:20988A000200BE06CE8C0200021005000000030F80010000040F05430000050F3A1A02002D
:2098AA00BE06CF8C0200021006000000030FA0010000040F06430000050F3A1A0200BE0628
:2098CA00D08C0200021007000000030FC0010000040F07430000050F3A1A0200BE06D18C4C
:2098EA000200021008000000030FE0010000040F08430000050F3A1A0200BE06D28C020063
:20990A00021009000000030F00020000040F09430000050F3A1A0200BE06D38C020002100E
:20992A000A000000030F20020000040F0A430000050F3A1A0200BE06D48C020002100B00D2
:20994A000000030F40020000040F0B430000050F3A1A0200BE06D58C020002100C00000099
:20996A00030F60020000040F0C430000050F3A1A0200BE06D68C020002100D000000030F44
:20998A0080020000040F0D430000050F3A1A0200BE06D78C020002100E000000030FA00271
:2099AA000000040F0E430000050F3A1A0200BE06D88C020002100F000000030FC0020000B0
:2099CA00040F0F430000050F3A1A0200BE06D98C0200021010000000030FE0020000040F5A
:2099EA0010430000050F3A1A0200BE06DA8C0200021011000000030F00030000040F1143D5
:209A0A000000050F3A1A0200BE06DB8C0200021012000000030F20030000040F12430000E4
:209A2A00050F3A1A0200BE06DC8C0200021013000000030F40030000040F13430000050F8D
:209A4A003A1A0200BE06DD8C0200021014000000030F60030000040F14430000050F3A1A0A
:209A6A000200BE06DE8C0200021001000000030F80030000040F15430000050F541A020013
:209A8A00BE06DF8C0200021002000000030FA0030000040F16430000050F541A0200BE060E
:209AAA00E08C0200021003000000030FC0030000040F17430000050F541A0200BE06E18C22
:209ACA000200021004000000030FE0030000040F18430000050F541A0200BE06E28C020049
:209AEA00021005000000030F00040000040F19430000050F541A0200BE06E38C02000210F5
:209B0A0006000000030F20040000040F1A430000050F541A0200BE06E48C020002100700BC
:209B2A000000030F40040000040F1B430000050F541A0200BE06E58C02000210080000007F
:209B4A00030F60040000040F1C430000050F541A0200BE06E68C0200021009000000030F2A
:209B6A0080040000040F1D430000050F541A0200BE06E78C020002100A000000030FA00455
:209B8A000000040F1E430000050F541A0200BE06E88C020002100B000000030FC004000096
:209BAA00040F1F430000050F541A0200BE06E98C020002100C000000030FE0040000040F40
:209BCA0020430000050F541A0200BE06EA8C020002100D000000030F00050000040F2143AB
:209BEA000000050F541A0200BE06EB8C020002100E000000030F20050000040F22430000CB
:209C0A00050F541A0200BE06EC8C020002100F000000030F40050000040F23430000050F73
:209C2A00541A0200BE06ED8C0200021010000000030F60050000040F24430000050F541AD6
:209C4A000200BE06EE8C0200021011000000030F80050000040F25430000050F541A0200FF
:209C6A00BE06000000003E0AFF0000000C0F2C0C04003E01CE9D0200140F00000092CF70D8
:209C8A00000000203F04000000043E598E9D0200140F000000203F04000000003E59000072
:209CAA00008A0F7001000000240F0E9E0200100F00000000300F000000B48F700A00000094
:209CCA001E0E000000003E59000000803E51000000003E59000000803E51000000003E596B
:209CEA00000000803E51000000003E59000000803E51000000003E59000000803E5100FF00
:209D0A0000000C0F2C0C04003E01CCF800783E02CE9D0200140F00000092CF7000000020A6
:209D2A003F04000000063E598C1800003E018E9D0200140F000000203F04000000003E590C
:209D4A000000008A0F7001000000240F000000B4CF700A0000001E0E000000003E590000FC
:209D6A0000803E51000000003E59000000803E51000000003E59000000803E51000000007E
:209D8A003E59000000803E51000000003E59000000803E51000000003E0A00A302003E0141
:209DAA00010070000411071A0200BE060E9E0200140F01000000240F000000000C0F00000C
:209DCA0000B48F70030000001E0E000000003E59000070000011000070000C110100700081
:209DEA0005110000700008113A8C0200140F000000923F7000000000340F000000203F04E8
:209E0A0000000000240F000000003E5900000100010F010004003E01FFFF0000010F1202F7
:209E2A0004003E01021004003E01000000803E59000000003E0A00A302003E0101007000CC
:209E4A000411071A0200BE060E9E0200140F01000000240F000000000C0F000000B48F7029
:209E6A00030000001E0E000000003E59000070000011000070000C1101007000051100007D
:209E8A00700008114E8C0200140F000000923F7000000000340F000000203F040000000049
:209EAA00240F000000003E5900000100010F010004003E01FFFF0000010F120204003E0114
:209ECA00021004003E01000000803E59000000003E0A20410000010F0100700001110000D0
:209EEA007000031123410000010F01007000011100007000041126410000010F0100700070
:209F0A00011100007000051129410000010F0100700001110000700006112C410000010F9E
:209F2A00010070000111000070000711000000003E0A00000000300F01000000200F000055
:209F4A000000310F7FEE0200221000000000320F83A10200130F00000000330F71A1020037
:209F6A002310B0ED0200140F00000000340F54EE0200150F00000000350F00000000250FBF
:209F8A0052EC0200160F00000000360F69EE0200170F00000000370F000000003A0F0000FF
:209FAA0000003B0F000000003C0F000000003D0F000000003E0F000042001F0F00000000F9
:209FCA003F0F010000002C0FCAA102002D107BA102002E10800000002F0F6CA102000B10FF
:209FEA006DA102000E1000000000050F143802000511FF2F84013E56553802001D0F0000AF
:20A00A00008DFF717FEE020006103FC02C003E01AB1A020410060000008EDF71F09F0230CA
:20A02A007F040000008FFF71000000B07F0402000000060D000000023F5D000000823F5994
:20A04A00000000687F04FB2C00E87F04A21A0200020671A1020006107FA102000C10C01C6F
:20A06A0002003E01B71A020000060000008EDF710000008FFF7102000000060D00000002C8
:20A08A003F5D000000823F59000000787F04000000F87F0480A102000C10C01C02003E012E
:20A0AA00C11A020000060000008EDF710000008FFF7102000000060D000000023F5D000023
:20A0CA0000823F59000000787F04000000F87F0481A102000C10C01C02003E01CB1A0200A2
:20A0EA0000060000008EDF710000008FFF7102000000060D000000023F5D000000823F59A6
:20A10A00000000787F04000000F87F0482A102000C10C01C02003E01D51A0200000600006A
:20A12A00008EDF710000008FFF7102000000060D000000023F5D000000823F59000000F873
:20A14A007F04FF2F04003E01553802001D0F80EE020002107EEE0200061015B80200110F51
:20A16A0000000000080FCDCCCC3D090F3FC02C003E01EC1A020410060000008EDF71F09F0B
:20A18A0002307F04000000881F71000000891F71DD2D84033E50CC2C04220124020000006B
:20A1AA00060D35D9D8033E5000C85822012400C858003E018C1808003E0135D958003E01B5
:20A1CA009D1908003E01000000687F04FB2C00503E04DD1A020002067FA102000C10C01CB9
:20A1EA0002003E01FE1A02000006000000881F71000000891F710000008EDF71DD2D840354
:20A20A003E50CC2C0422012402000000020D35D9D8033E5000C85822012400C858003E0115
:20A22A008C1808583E0435D958003E019D1908003E01000000787F0480A102000C10C01C16
:20A24A0002003E010E1B02000006000000881F71000000891F710000008EDF71DD2D8403E2
:20A26A003E50CC2C0422012402000000020D35D9D8033E5000C85822012400C858003E01B5
:20A28A008C1808583E0435D958003E019D1908003E01000000787F0481A102000C10C01CB5
:20A2AA0002003E011E1B02000006000000881F71000000891F710000008EDF71DD2D840372
:20A2CA003E50CC2C0422012402000000020D35D9D8033E5000C85822012400C858003E0155
:20A2EA008C1808583E0435D958003E019D1908003E01000000787F0482A102000C10C01C54
:20A30A0002003E012E1B02000006000000881F71000000891F710000008EDF71DD2D840301
:20A32A003E50CC2C0422012402000000020D35D9D8033E5000C85822012400C858003E01F4
:20A34A008C1808583E0435D958003E019D1908003E01000080869F70ECA102000010000057
:20A36A000040090FD0408C830F700D0D13003E01357059003E010D0D13003E0135705900CA
:20A38A003E010D0D13003E01357059003E01070713003E01000080833E580000A040000FE3
:20A3AA00000080808F7080380E003E01812108003E014E1B02040006000000027E5B020054
:20A3CA0000000C0F409402003E014C2C00003E01531B020402060000003F020F00000000C0
:20A3EA00000000000001001468EE0200041045042C003E0168EE02000411CDCCCC3D020FFE
:20A40A00531B02043E06442404003E0100000000000040A402003E01531B0204220672F9A3
:20A42A007F3F020F00000000000000000000040F000000823E5A000000003E5C0824080048
:20A44A003E01000000823E5E0000080080145A1B02001A0600000000030F553802001D0F95
:20A46A00553E02001B0F7FEE02000610FF2F04003E0115B80200110F470513003E013FC091
:20A48A002C003E01701B020410060000008EDF71F09F02307F04000008008014701B020055
:20A4AA003A060000008FBF71000000B07F04000000881F71000000220120240C13003E0183
:20A4CA0005091322012084C858003E0102000000060D05091322012084C858843F5D0000EE
:20A4EA0000687F04000000E87E04FB2C00503E04601B02000206000010008014B51B020049
:20A50A003A0671A1020006107FA102000C10C01C02003E01851B020000060000008EDF71E6
:20A52A000000008FBF71000000881F71000000220120240C13003E0105091322012084C8C5
:20A54A0058003E0102000000060D05091322012084C858843F5D000000583E04000000780B
:20A56A007F04000000F87E0480A102000C10C01C02003E01951B020000060000008EDF71E2
:20A58A000000008FBF71000000881F71000000220120240C13003E0105091322012084C865
:20A5AA0058003E0102000000060D05091322012084C858843F5D000000583E0400000078AB
:20A5CA007F04000000F87E0481A102000C10C01C02003E01A51B020000060000008EDF7171
:20A5EA000000008FBF71000000881F71000000220120240C13003E0105091322012084C805
:20A60A0058003E0102000000060D05091322012084C858843F5D000000583E04000000784A
:20A62A007F04000000F87E0482A102000C10C01C02003E01B51B020000060000008EDF71FF
:20A64A000000008FBF71000000881F71000000220120240C13003E0105091322012084C8A4
:20A66A0058003E0102000000060D05091322012084C858843F5D000000583E04FF2F040030
:20A68A003E01553E02001D0F7FEE020006103FC02C003E01C11B020410060000008EDF71EB
:20A6AA00F09F02307F040000008FAF71000000B07F0402000000060D000000023F590000BB
:20A6CA0000823F5D000000687F04FB2C00A87E04B81B02000206000010008014ED1B02008B
:20A6EA003A0671A1020006107FA102000C10C01C02003E01CF1B020000060000008EDF71BB
:20A70A000000008FAF7102000000060D000000023F59000000823F5D000000787F040000B8
:20A72A0000B87E0480A102000C10C01C02003E01D91B020000060000008EDF710000008F10
:20A74A00AF7102000000060D000000023F59000000823F5D000000787F04000000B87E04CD
:20A76A0081A102000C10C01C02003E01E31B020000060000008EDF710000008FAF710200DD
:20A78A000000060D000000023F59000000823F5D000000787F04000000B87E0482A102008A
:20A7AA000C10C01C02003E01ED1B020000060000008EDF710000008FAF7102000000060DA4
:20A7CA00000000023F59000000823F5D143802000510509502003E011438020005115E214B
:20A7EA0000003E019E1A02000206000000003E0A4DEC02000010B8EE020000110100000001
:20A80A00200F00000000210F02EE0200100F00000000300F19EE0200140F00000000340F10
:20A82A00DAED0200150F00000000350F00000000360F16EE020003104FEC02000A10000028
:20A84A0000000F0FB7EE02000F116CA102006810280000001E0EAFC02C003E01271C02000F
:20A86A0030063FC02C003E011F1C02041006000000007E5000A102003E01000000003F04E4
:20A88A004FEE020001101F012C003E014FEE02000111009002003E0103000000010F01217C
:20A8AA0000003E011C1C020402063F432C003E0116EE02000311000020000014B7EE020027
:20A8CA0000100F002C003E01B7EE0200001100000000020F2B1C02043E0600000000000F7B
:20A8EA00000000803E502B1C02043E06000000803E50CDCC4C3E020F211C02000206000026
:20A90A0080807E50000000003E0450EC02000210F09F02003E012000000080145E1D0200CC
:20A92A009A062B1C02003E06000000003E04000000003F04F09F02003E0100000000020F7A
:20A94A00000000813E5A18EE02000C1020000000040FC42C00003E01321C020002060000F6
:20A96A000000000F18EE020000110400000080143A1C02003A06DAED0200150FA3EE0200F5
:20A98A00160F6CA102006810020000001E0E000000003E5A000000803E5C00000000310FE1
:20A9AA002FEE0200120F00000000320F83A10200130F00000000330F7BA1020023107BA115
:20A9CA000200271000A00000380F00604200480F01000000280FCBA1020029100000000075
:20A9EA002C0F000000003C0F000042001D0F000000003D0FCAA102002D107BA102002E1007
:20AA0A00000000003E0F000000707F0400A000003F0F006042004F0F000043001F1050EE4E
:20AA2A0002000A1078A1020005105A2F00003E01551C02002406000000855F700000000007
:20AA4A00050F5A2500003E01000080955F70000000D87F04000043001F11800000002F0FAA
:20AA6A0000000000050FA2EE020005117EEE020006106CA1020009106DA102000E10FF2F08
:20AA8A0084013E5697A10200140F3FC02C003E01791C020010064FEC020008108FC02C004F
:20AAAA003E01791C02003006000000003E5800A002003E01000080920F70000000007E45B5
:20AACA00000080880F70000000B4AF700000008EDF710000008CFF71080000001E0E882854
:20AAEA0004020122CC2C84831F7101000000060D00C85802012200C858003E018C18888828
:20AB0A007F700000008EDF71000000843F507E1C02003E06000000003F04000000B4AF7055
:20AB2A000000008CFF71010000001E0E000000002090F09F02687F04F92C00C87F04621CC8
:20AB4A0002000206000000787F04000000787F04000000787F04000000787F04A2EE020063
:20AB6A000510509502003E01A2EE020005115E2100003E01601C0200020670EC0200100F27
:20AB8A0083A10200130F52EC0200170F00000000370F00000000390F00000000380F000028
:20ABAA0000003D0F00A000003C0F006042004C0F00A000003E0F006042004E0F0000430028
:20ABCA001E1000000000050FA2EE020005116CA1020009106DA102000E10A7A10200120FC0
:20ABEA00DAED0200150FFF2F84013E56000000053E5E00300200190F3FC02C003E01C61CD0
:20AC0A0002041006000000017E5A4FEC020008108FC02C003E01C61C02003006CDCCCC3D6A
:20AC2A000D0F00000000000F000080007E501A0113003E010000008EEF71B7EE0200081077
:20AC4A008FC02C003E01B01C020410060000008C9F710000808E9F7100000000010F00007E
:20AC6A0000347E54000000023F50050000001E0E240C13043F58180513023F50C52C08006A
:20AC8A003E01880013863F5A0D1D08003E01400000008014C41C02043A06EAA102000010A9
:20ACAA00000000400B0FD0408C830F700D0D13003E013D7059003E010D0D13003E013D70C8
:20ACCA0059003E010D0D13003E013D7059003E01070013003E01000000807E500000803FBB
:20ACEA00020F000000003E04000000803E04000000813E5AF09F02487E04F92C00887F0491
:20AD0A009F1C02000206A2EE02000510509502003E01A2EE020005115E2100003E019A1C7B
:20AD2A0002000206040000008014591D02003A0683A10200130F00A00000380F020043003B
:20AD4A00480F000000003C0F000042001D0F000000003E0F000000707F0400A000003F0FAB
:20AD6A00020043004F0F02A043001F1050EE02000A1079A1020005105A2F00003E01E21CC1
:20AD8A0002002406000000855F7000000000050F5A2500003E01000080955F70000000D89B
:20ADAA007F0402A043001F1100000000050FA2EE020005117EEE020006106CA10200091089
:20ADCA006DA102000E10FF2F84013E5633EE0200120F3FC02C003E01021D020010064FECD4
:20ADEA00020008108FC02C003E01021D02003006000000003E54000080880F70000000B451
:20AE0A00AF700000008EDF710000008CFF71080000001E0E882804020122CC2C84831F7193
:20AE2A0001000000060D00C85802012200C858003E018C1888887F700000008EDF710000CF
:20AE4A0000843F50071D02003E06000000803E04000000B4AF700000008CFF7101000000D9
:20AE6A001E0E000000002090F09F02687F04F92C00C87F04EE1C02000206000000787F04F1
:20AE8A00000000787F04000000787F04000000787F04A2EE02000510509502003E01A2EE5A
:20AEAA00020005115E2100003E01EC1C0200020610ED0200100F83A10200130F52EC0200FA
:20AECA00170F00A000003C0F020043004C0F00A000003E0F020043004E0F02A043001E1015
:20AEEA0000000000050FA2EE020005116CA1020009106DA102000E10A3EE0200150FB7A127
:20AF0A000200120FFF2F84013E56000000053E5E00340200190FDAED0200150F3FC02C00A6
:20AF2A003E014E1D02041006000000017E5A4FEC020008108FC02C003E014E1D02003006B6
:20AF4A00CDCCCC3D0D0F00000000000F000080007E501A0113003E010000008EEF71B7EECC
:20AF6A00020008108FC02C003E01361D020410060000008C9F710000808E9F7100000000CA
:20AF8A00010F000000347E54000000023F50050000001E0E240C13043F58180513023F5030
:20AFAA00C52C08003E01880013863F5A0D1D08003E01EAA1020000104000000080144C1D4A
:20AFCA0002043A060000803E0B0F0B0013003E01000000400B0FD0408C830F700D0D1300C7
:20AFEA003E013D7059003E010D0D13003E013D7059003E010D0D13003E013D7059003E0161
:20B00A00070013003E01000000807E500000803F020F000000003E04000000813E5A000054
:20B02A0000803E04F09F02487E04F92C00887F04251D02000206A2EE0200051050950200DF
:20B04A003E01A2EE020005115E2100003E011F1D020002064FEC02000010B7EE02000110F6
:20B06A00000000043E0A011004003E014FEC0200001118EE02000C1020000000040FC42499
:20B08A0000003E01761D02000206000000007E586F12833A010F000080803E58C0AC0C0098
:20B0AA003E01000000400B0FC0408C830F700C0C13003E013C7059003E010C0C13003E0147
:20B0CA003C7059003E010C0C13003E013C7059003E01070013003E01EAA102000110EBA1F1
:20B0EA0002000410100113003E01140113003E01000000043E0A0000803F040F41220800DD
:20B10A003E01000000043E0A000000017E5A000000000000AAAAAAAA000F68EC02000011A3
:20B12A0069EC020000116AEC02000011EC1D0200BE06AA8C0200001000000000010F0121EB
:20B14A0000003E01E61D0200000601000000240F00000000340F00005000150F00000000B0
:20B16A00350F00000000380F01000000280F000000003E5B000010103E02A5000000030F52
:20B18A00032000003E01A91D02002006C48C0200140F80000000680FBB1F0200BE06B48C09
:20B1AA000200140F10000000680FBB1F0200BE066AA10200140F80000000680FBB1F020036
:20B1CA00BE06EAA10200140F10000000680FBB1F0200BE0600004200180F00600000680F8A
:20B1EA00CD1F0200BE0600300200180F00040000680FCD1F0200BE0600340200180F0004AC
:20B20A000000680FCD1F0200BE06A5E70200140FBC000000680FBB1F0200BE06F9E3020099
:20B22A00140FAC030000680FBB1F0200BE0614170200BE06AA8C0200001000000000010FD2
:20B24A00012100003E01E61D02000006AA8C0200001002000000010F012100003E01C31DDD
:20B26A00020020060A000000000F928C02000011B08C0200001002000000010F01210000D0
:20B28A003E01BA1D02002006D41D02043E0602000000001401000000001403000000010FED
:20B2AA00012100003E01C01D02002006D41D02043E06020000002014010000000014D41DA7
:20B2CA0002043E06020000000014010000002014AB8C0200001003000000010F1021000042
:20B2EA003E01CA1D0200200601000000000F928C02000011D41D02003E0602000000010F6C
:20B30A00102100003E01D21D020020060A000000000F928C02000011D41D02043E06020015
:20B32A000000201401000000201400000000000F928C02000011AF8C02000010000000000D
:20B34A00010F012100003E01DD1D0200200601000000000F8A8C02000011E61D02043E06CA
:20B36A0000000000000F918C0200001100000000010F8A8C0200011103000000010F012115
:20B38A0000003E01E61D0204000601000000000F918C0200001101000000000F8A8C0200ED
:20B3AA00001100000000000F68EC0200001169EC020000116AEC02000011EC1D0200BE065C
:20B3CA00000000003E0A000010000C140A00000000000800ED1D02000E00000000000100BE
:20B3EA00F51D0200000010002C140A00000000000800F61D02000E00000000000100FE1D8E
:20B40A000200000020002C140A00000000001000FF1D02000E00000000000A000F1E020041
:20B42A0000000000000F000008008C14131E02003A0601000000000F6AEC0200031000005D
:20B44A0000000F0F000040002C143FC02C003E01191E02001006000040000C140A00000021
:20B46A0000000800191E02000E00000000000100211E0200000020000C140A0000000000E7
:20B48A000800221E02000E000000000001002A1E0200000020002C140A0000000000100085
:20B4AA002B1E02000E00000000000A003B1E0200000008008C143F1E02003A0600900200EB
:20B4CA003E01009002003E01AA8C02000011000040002C14F09F02003E013FC02C003E014F
:20B4EA00451E02001006000040000C140A00000000000800451E02000E00000000000100E1
:20B50A004D1E0200000020000C140A000000000008004E1E02000E00000000000100561E71
:20B52A000200000020002C140A00000000001000571E02000E00000000000900671E020070
:20B54A0000000000000F000008008C146B1E02003A0601000000000FF09F02003E0100007F
:20B56A0040002C143FC02C003E01701E02001006000040000C140A00000000000800701E31
:20B58A0002000E00000000000100781E0200000020000C140A00000000000800791E02000D
:20B5AA000E00000000000100811E0200000020002C140A00000000001000821E02000E00A7
:20B5CA00000000000A00921E0200000008008C14961E02003A06009002003E0100900200A4
:20B5EA003E01AB8C02000011000040002C14F09F02003E013FC02C003E019C1E020010062C
:20B60A00000040000C140A000000000008009C1E02000E00000000000100A41E020000001F
:20B62A0020000C140A00000000000800A51E02000E00000000000100AD1E020000002000ED
:20B64A002C140A00000000001000AE1E02000E00000000000900BE1E020000000000000FB4
:20B66A00000008008C14C21E02003A0601000000000FF09F02003E01000040002C143FC097
:20B68A002C003E01C71E02001006000040000C140A00000000000800C71E02000E000000D1
:20B6AA0000000100CF1E0200000020000C140A00000000000800D01E02000E000000000040
:20B6CA000100D81E0200000020002C140A00000000001000D91E02000E00000000000A00DC
:20B6EA00E91E0200000008008C14ED1E02003A06009002003E01009002003E01AF8C020063
:20B70A000011000040002C14F09F02003E013FC02C003E01F31E02001006000040000C14CB
:20B72A000A00000000000800F31E02000E00000000000100FB1E0200000020000C140A0066
:20B74A00000000000800FC1E02000E00000000000100041F0200000020002C140A0000001D
:20B76A0000001000051F02000E00000000000900151F020000000000000F000008008C1485
:20B78A00191F02003A0601000000000FF09F02003E01000040002C143FC02C003E011E1F1E
:20B7AA0002001006000040000C140A000000000008001E1F02000E00000000000100261F62
:20B7CA000200000020000C140A00000000000800271F02000E000000000001002F1F020064
:20B7EA00000020002C140A00000000001000301F02000E00000000000A00401F02000000FB
:20B80A0008008C14441F02003A06009002003E01009002003E01B08C0200001100004000A0
:20B82A002C14F09F02003E013FC02C003E014A1F02001006000040000C140A000000000099
:20B84A0008004A1F02000E00000000000100521F0200000020000C140A0000000000080097
:20B86A00531F02000E000000000001005B1F0200000020002C140A000000000010005C1FCA
:20B88A0002000E000000000008006C1F0200821F02003E0604000000680F130000001E0E58
:20B8AA00000040002C14F09F02003E013FC02C003E01741F02001006000040000C140A00AF
:20B8CA00000000000400741F02000E00000000000100781F0200000020000C140A000000D3
:20B8EA0000000400791F02000E000000000001007D1F0200000020002C140A000000000089
:20B90A0004007E1F02000E00000000000900821F0200FFFFFFFF0F0F69EC02000310140028
:20B92A000000680F130000001E0E000040002C14F09F02003E013FC02C003E018B1F0200E1
:20B94A001006000040000C140A000000000004008B1F02000E000000000001008F1F0200EE
:20B96A00000020000C140A00000000000400901F02000E00000000000100941F02000000FA
:20B98A0020002C140A00000000000400951F02000E00000000000900991F0200FFFFFFFFAC
:20B9AA000F0F68EC0200031014000000680F130000001E0E000040002C14F09F02003E01DC
:20B9CA003FC02C003E01A21F02001006000040000C140A00000000000400A21F02000E00DB
:20B9EA00000000000100A61F0200000020000C140A00000000000400A71F02000E00000051
:20BA0A0000000100AB1F0200000020002C140A00000000000400AC1F02000E000000000006
:20BA2A000100B01F0200000010000C140A00000000000400B11F02000E000000000001000B
:20BA4A00B51F0200000010002C140A00000000000400B61F02000E00000000002500BA1FC5
:20BA6A000200000000003E0A100000001E0E000000003E5B000010103E0210F802783E027B
:20BA8A00000000003E5B000010103E02101100003E0111F802783E02000000003E5B0000E7
:20BAAA0010103E02101100003E0111F802783E02000000003E5B000010103E0210110000DF
:20BACA003E0111F802783E02000080803E59000000003E0A100000001E0E000000003E5BA6
:20BAEA00000010103E0210F802783E02000000003E5B000010103E02101100003E0111F8B8
:20BB0A0002783E02000000003E5B000010103E02101100003E0111F802783E020000000045
:20BB2A003E5B000010103E02101100003E0111F802783E02000080803F50000000003E0A08
:20BB4A000800000000005514003002000200000000008A1D00800200050000000000030005
:20BB6A008A9D0200000000100000000000000000000000100000020000000000AA008D9D9C
:20BB8A0002000500000000000100379E02000000FF3F00000200000000001300389E020091
:20BBAA0005000000000010004B9E02000000010000000000AC040000000017F900000000BA
:20BBCA00AC040000000052BE00000000DCEA000000007D120000000069FF000000007D124F
:20BBEA00000000005FC30000000099DA000000007B2300000000FD0F000000007B2300005E
:20BC0A00000030C5000000005FCA000002000000000005005B9E02000500000000001000E5
:20BC2A00609E020000000300000000004709000000006AEF00000000470900000000CFDE51
:20BC4A0000000000E7F500000000B41900000000A4E700000000B4190000000079F100006F
:20BC6A000000F0DF000000008A290000000081E9000000008A2900000000DEFD0000000040
:20BC8A004DCD00000200000000000500709E02000500000000001000759E0200000003003C
:20BCAA0000000000320D000000002DE700000000320D00000000C9F2000000002BF9000009
:20BCCA000000D71E000000005AD600000000D71E00000000E30D0000000028E00000000048
:20BCEA001E2D0000000084D0000000001E2D000000002F1F0000000078CD000002000000BB
:20BD0A0000000500859E020005000000000010008A9E02000000030000000000C90F0000D5
:20BD2A0000006BE100000000C90F00000000D7FD00000000ECF90000000078210000000083
:20BD4A00B5C900000000782100000000E51E00000000E7DF000000009F2E000000001BBE53
:20BD6A00000000009F2E00000000BE330000000000CD000002000000000005009A9E0200ED
:20BD8A0005000000000010009F9E0200000003000000000091150000000036D50000000091
:20BDAA00911500000000C71B00000000C4F70000000063240000000018BB00000000632455
:20BDCA0000000000C43B0000000001E000000000532C0000000022AF00000000532C0000AA
:20BDEA0000003E4C00000000ADD200000200000000000500AF9E02000500000000001000C5
:20BE0A00B49E020000000300000000003E1A00000000A2CB000000003E1A00000000E52E91
:20BE2A0000000000EAF0000000007A240000000036B8000000007A240000000000450000AF
:20BE4A00000021DF0000000071280000000049B1000000007128000000000F4E000000004F
:20BE6A007DD700000200000000000500C49E02000500000000001000C99E02000000030078
:20BE8A0000000000711A0000000040CB00000000711A000000008E2D00000000FFF10000CC
:20BEAA00000020260000000015B50000000020260000000018470000000002DE00000000E3
:20BECA00FD2A0000000092AC00000000FD2A00000000255200000000DBD4000002000000A4
:20BEEA0000000500D99E02000500000000001000DE9E02000000030000000000711A000099
:20BF0A00000040CB00000000711A000000008E2D00000000FFF10000000020260000000090
:20BF2A0015B50000000020260000000018470000000002DE00000000FD2A0000000092AC43
:20BF4A0000000000FD2A00000000255200000000DBD400000200000000000500EE9E0200F5
:20BF6A000500000000001000F39E02000000030000000000711A0000000040CB0000000076
:20BF8A00711A000000008E2D00000000FFF10000000020260000000015B50000000020260B
:20BFAA000000000018470000000002DE00000000FD2A0000000092AC00000000FD2A0000AC
:20BFCA000000255200000000DBD400000200000000000500039F0200050000000000100071
:20BFEA00089F0200000003000000000046280000000008B0FFFF0000462800000000FB48B6
:20C00A000000000076E8FFFF0000B835000000003E99FFFF0000B83500000000A562000004
:20C02A00000073D0FFFF0000D33C000000008A8EFFFF0000D33C00000000BF6F0000000053
:20C04A00E8C3FFFF0200000000000500189F020005000000000010001D9F02000000030097
:20C06A000000000043220000000079BBFFFF0000432200000000A6380000000098EFFFFF57
:20C08A000000E13200000000FD9AFFFF0000E13200000000175F0000000091D3FFFF000003
:20C0AA005F3A00000000418BFFFF00005F3A0000000054710000000020C5FFFF02000000D0
:20C0CA00000005002D9F02000500000000001000329F02000000030000000000662400000E
:20C0EA00000034B7FFFF0000662400000000BD3E0000000025EDFFFF00004A34000000003A
:20C10A006C97FFFF00004A34000000001D6300000000F5D1FFFF0000133B00000000DA89A1
:20C12A00FFFF0000133B00000000AA7300000000A2C4FFFF0200000000000500429F02003E
:20C14A000500000000008E00479F020000000300000000000C2100000000E7BDFFFF000088
:20C16A000C210000000047350000000014F1FFFF0000AF3100000000A19CFFFF0000AF310E
:20C18A0000000000A15C00000000E3D5FFFF00008D3900000000E58CFFFF00008D390000E7
:20C1AA000000096F00000000D3C8FFFF0000743C000000001787FFFF0000743C0000000068
:20C1CA0014770000000076C2FFFF00000400000000007C250000000008B5FFFF00007C2593
:20C1EA0000000000E74100000000F6EBFFFF00009F3400000000C296FFFF00009F34000032
:20C20A000000CA64000000004ED2FFFF00001E3B00000000C489FFFF00001E3B00000000CB
:20C22A00A0730000000029C7FFFF0000483D000000006F85FFFF0000483D00000000F2798C
:20C24A0000000000F9C1FFFF0000040000000000BA28000000008CAEFFFF0000BA2800001C
:20C26A000000A24A00000000BBE7FFFF0000843600000000F892FFFF00008436000000002C
:20C28A00D76900000000C6CFFFFF00000F3C00000000E287FFFF00000F3C00000000497605
:20C2AA00000000000DC6FFFF0000BF3D000000008184FFFF0000BF3D00000000807B0000AD
:20C2CA000000A7C1FFFF00000400000000002E2D00000000A3A5FFFF00002E2D00000000EE
:20C2EA000B560000000051E1FFFF0000D53800000000558EFFFF0000D53800000000C46F75
:20C30A00000000006ECCFFFF0000233D00000000B985FFFF0000233D000000003679000030
:20C32A000000A8C4FFFF00003D3E000000008583FFFF00003D3E000000001A7D00000000F6
:20C34A0042C1FFFF00000400000000006A30000000002B9FFFFF00006A3000000000EE5D87
:20C36A000000000044DCFFFF0000563A00000000548BFFFF0000563A0000000073730000B2
:20C38A0000001ACAFFFF0000CC3D000000006784FFFF0000CC3D00000000EC7A0000000050
:20C3AA00BAC3FFFF0000843E00000000F782FFFF0000843E00000000F77D0000000000C1C8
:20C3CA00FFFF0000040000000000FD34000000000596FFFF0000FD3400000000926800005C
:20C3EA0000009CD4FFFF00003E3C000000008387FFFF00003E3C00000000EE770000000064
:20C40A00F3C6FFFF0000973E00000000D282FFFF0000973E00000000E17C0000000084C2BC
:20C42A00FFFF0000D23E000000005B82FFFF0000D23E00000000DE7E00000000ACC0FFFF33
:20C44A0000000400000000006A39000000002C8DFFFF00006A39000000005372000000000C
:20C46A00ACCCFFFF0000003E00000000FF83FFFF0000003E00000000CD7B00000000CAC36B
:20C48A00FFFF0000C53E000000007682FFFF0000C53E00000000DD7E00000000E1C0FFFF9E
:20C4AA000200000000000500D59F02000500000000001000DA9F0200000003000000000062
:20C4CA00270D00000000A01900000000270D00000000840400000000BFFA00000000241CB0
:20C4EA00000000002E2F00000000241C0000000002E700000000B6E400000000B827000033
:20C50A000000E63A00000000B8270000000094D300000000ABD30000020000000000050026
:20C52A00EA9F02000500000000001000EF9F02000000030000000000080800000000DE0EC2
:20C54A000000000008080000000082250000000024F500000000FD1500000000DB190000FB
:20C56A000000FD1500000000D11100000000F1E1000000009D2400000000A61C0000000068
:20C58A009D240000000081030000000006CF00000200000000000500FF9F020005000000CB
:20C5AA000000100004A0020000000300000000003905000000001D09000000003905000016
:20C5CA00000096360000000070EF00000000F01000000000770C00000000F01000000000A3
:20C5EA00602B00000000E0DF00000000411F00000000950700000000411F00000000F9236F
:20C60A0000000000B6CE0000020000000000050014A00200050000000000100019A00200FF
:20C62A000000030000000000570500000000510900000000570500000000CD3700000000D7
:20C64A0012EF00000000501100000000BE0C00000000501100000000572C0000000029DFB8
:20C66A0000000000F31F00000000C00700000000F31F00000000C624000000009DCD000071
:20C68A00020000000000050029A0020005000000000010002EA002000000030000000000D6
:20C6AA003D03000000009504000000003D0300000000CB4900000000A7E600000000360E72
:20C6CA000000000019FE00000000360E00000000304700000000CCD900000000431D000079
:20C6EA00000092ED00000000431D0000000092470000000060CB0000020000000000050046
:20C70A003EA00200050000000000100043A0020000000300000000009D020000000054033C
:20C72A00000000009D0200000000AE51000000008CE200000000E90C00000000E2FA000012
:20C74A000000E90C0000000013510000000000D700000000B81B000000000AE800000000DA
:20C76A00B81B00000000485300000000ABC90000020000000000050053A0020005000000CC
:20C78A000000100058A0020000000300000000003A02000000007C02000000003A0200008C
:20C7AA000000F9560000000083DF000000003A0C000000005AF8000000003A0C00000000E0
:20C7CA00BA5700000000E5D400000000F81A0000000093E300000000F81A00000000145B7C
:20C7EA00000000008BC80000020000000000050068A0020005000000000010006DA00200A7
:20C80A0000000300000000000C0200000000D301000000000C0200000000015B00000000BF
:20C82A0024DD000000009D0C00000000F9F4000000009D0C00000000FF5C00000000E0D2A1
:20C84A0000000000141C000000001BDD00000000141C0000000036610000000059C70000BF
:20C86A0002000000000005007DA00200050000000000100082A0020000000300000000004C
:20C88A00980100000000F70000000000980100000000B96100000000D3D800000000770B1E
:20C8AA000000000014F300000000770B00000000A0640000000012D0000000006D1A000078
:20C8CA00000028DA000000006D1A000000007C69000000000CC60000020000000000050007
:20C8EA0092A00200050000000000100097A0020000000300000000006B01000000005600E7
:20C90A00000000006B010000000060650000000027D600000000CB0B00000000F7EF000023
:20C92A000000CB0B0000000000690000000028CE000000004B1B000000008FD400000000EF
:20C94A004B1B00000000176E0000000058C500000200000000000500A7A002000500000070
:20C96A0000001000ACA0020000000300000000003F01000000000000000000003F010000CC
:20C98A000000CD6800000000BCD300000000600B000000002BEF00000000600B00000000D9
:20C9AA008C6C000000008FCC00000000AD1A000000005ED300000000AD1A00000000967154
:20C9CA00000000009EC400000200000000000500BCA002000500000000001000C1A002000E
:20C9EA0000000300000000001B0100000000BCFF000000001B0100000000566B0000000076
:20CA0A00BED100000000050B0000000093EE00000000050B00000000156F0000000054CB39
:20CA2A00000000001C1A0000000092D2000000001C1A00000000EF73000000003BC40000BB
:20CA4A000200000000000500D1A002000500000000001000D6A002000000030000000000C2
:20CA6A0013010000000079FF00000000130100000000096D0000000060D000000000720BE9
:20CA8A0000000000ECEC00000000720B00000000DD70000000005BCA00000000F21A0000B9
:20CAAA000000A5CF00000000F21A000000008A7500000000E1C30000020000000000050042
:20CACA00E6A002000500000000001000EBA002000000030000000000CA000000000070FFE6
:20CAEA0000000000CA00000000002871000000002BCD00000000620900000000B1EF0000C6
:20CB0A0000006209000000005974000000008AC80000000010170000000085D50000000000
:20CB2A001017000000007E78000000002CC300000200000000000500FBA002000500000036
:20CB4A000000100000A102000000030000000000E70000000000F5FE00000000E700000054
:20CB6A000000A4730000000042CB00000000780B00000000DCEA00000000780B00000000BB
:20CB8A00FA7600000000E7C600000000191B000000005FCC00000000191B00000000BB7AA6
:20CBAA000000000056C20000020000000000050010A10200050000000000100015A10200CC
:20CBCA0000000300000000009600000000003AFF00000000960000000000D4760000000099
:20CBEA0070C8000000004E080000000060F0000000004E08000000003379000000007DC509
:20CC0A0000000000E71400000000A6D700000000E71400000000367C00000000FDC1000027
:20CC2A00020000000000050025A1020005000000000010002AA10200000003000000000036
:20CC4A00130200000000130200000000000000000000843B00000000000000000000CB0313
:20CC6A0000000000F9F800000000CB0300000000CD780000000050C600000000AE0F0000D3
:20CC8A0000009AE100000000AE0F000000005A7C000000005AC20000020000000000050059
:20CCAA003AA1020005000000000010003FA10200000003000000000084000000000018FFF8
:20CCCA0000000000840000000000407B000000009FC40000000013080000000029F0000074
:20CCEA000000130800000000C37C00000000EFC200000000481400000000DFD7000000000D
:20CD0A00481400000000F77D0000000042C1000002000000000005004FA102000500000038
:20CD2A000000100054A102000000030000000000BE000000000096FE00000000BE000000CF
:20CD4A000000657C0000000088C300000000240B00000000E4E900000000240B0000000072
:20CD6A00BA7D000000001AC2000000002B1A00000000E6CB000000002B1A000000003A7EA3
:20CD8A000000000015C10000020000000000050064A10200050000000000010069A1020093
:20CDAA00000003000000020000000000B70B6AA10200050000000000010021AD02000000BF
:20CDCA0031A20200020000000000F10A22AD0200050000000000010013B80200000023AD03
:20CDEA000200020000000000F12014B80200050000000000010005D90200000015CE02007B
:20CE0A00020000000000F10A06D902000500000000000100F7E30200000015CE0200020061
:20CE2A00000000006E08F8E30200050000000000020066EC02000000010000000000010038
:20CE4A000000020000000000290268EC02000500000000000B0091EE02006E0083F9A23EEA
:20CE6A000000001049405D007A7715B7000000008035FD0038774FABBD00AA72302F8C00D6
:20CE8A00A531D7B2EF001BEF3836CD00000D50B989008888083CAB00AAAA2ABE0200000019
:20CEAA0000001E009CEE0200080000000000FCFF000042000800000000000400FCFF420030
:20CECA000C000000000001000000430000000060420008000000000001A0010043000C005D
:20CEEA0000000000020002A0430000000200430000000000000000000000000000000000FC
:20CF0A003E0B0000000000000000000000000000000000000000000000000020802D733945
:20CF2A005B1602003E06000000003E0B000000003E0B00000000000000000000000000009E
:20CF4A0000000000000000000000000000003E0B000000003E0B000000003E0B00000000EC
:20CF6A003E0B000000003E0B000000003E0B000000003E0B000000003E0B000000003E0BF1
:20CF8A00000000003E0B000000003E0B000000003E0B000000003E0B000000003E0B00001A
:20CFAA0000003E0B000000003E0B000000003E0B000000003E0B000000003E0B00000000FA
:20CFCA003E0B85000200BE06000000003E0B000000003E0B000000003E0B000000000000D8
:20CFEA00000000000000000000000000000000000000000000003E0B000000003E0B000095
:20D00A0000003E0B000000003E0B88070200BE06000000003E0B000000003E0B000000008D
:20D02A003E0B000000003E0B000000003E0B000000003E0B000000003E0B000000003E0B30
:20D04A00000000003E0B000000003E0B000000003E0B000000003E0B000000003E0B000059
:20D06A0000003E0B000000003E0B000000003E0B000000003E0B000000003E0B0000000039
:20D08A003E0B000000003E0B000000003E0B000000003E0B000000003E0B000000003E0BD0
:20D0AA00000000003E0B000000003E0B000000003E0B000000003E0B000000003E0B0000F9
:20D0CA0000003E0B000000003E0B000000003E0B000000003E0B000000003E0B00000000D9
:20D0EA003E0B000000003E0B000000003E0B000000003E0B000000003E0B000000003E0B70
:20D10A00000000003E0B000000003E0B000000003E0B000000003E0B000000003E0B000098
:20D12A0000003E0B000000003E0B000000003E0B000000003E0B000000003E0B0000000078
:20D14A003E0B000000003E0B000000003E0B000000003E0B000000003E0B000000003E0B0F
:20D16A00000000003E0B000000003E0B000000003E0B000000003E0B000000003E0B000038
:20D18A0000003E0B000000003E0B000000003E0B000000003E0B000000003E0B0000000018
:20D1AA003E0B000000003E0B000000003E0B000000003E0B000000003E0B000000003E0BAF
:20D1CA00000000003E0B000000003E0B000000003E0B000000003E0B000000003E0B0000D8
:20D1EA0000003E0B000000003E0B000000003E0B000000003E0B000000003E0B00000000B8
:20D20A003E0B000000000000000000000000000000000000000000000000000000000000BB
:20D22A00000400000B14800000000B14080000000B14200000000B14100000000B1400800D
:20D24A0002007C1100000000000F338C02000011328C02000110101102003E0150040200CB
:20D26A00000617EE02000010009002003E0117EE0200001101000000240FFFFFFFFF250F3A
:20D28A00010000002C0F000000003C0F928C020001100A000000000F012000003E01B4009F
:20D2AA0002002006BB8C0200001000940C003E01020000008014A90002003A0651EE020042
:20D2CA000110109102003E0151EE02000111110300003E02412000003E01A9000200220637
:20D2EA0000000004001400000000010F928C02000111B40002003E06010000008014B40087
:20D30A0002003A0653EE02000110109102003E0153EE02000111110300003E024120000081
:20D32A003E01B4000200220600000004001400000000010F928C0200011100000000340F29
:20D34A0040410000010F01007000011100000000000F001002003E01C100020400060EEC88
:20D36A000200140F163802001C0F01000000000F001002003E01C1000200200618EC0200B3
:20D38A00140F203802001C0FE1FFFFFF0C0FCDCCCC3D040FFFFFFFFF0F0F7DEE0200031093
:20D3AA000A000000680F0A0000001E0E000070000110111001003E021CA00D003E010002BF
:20D3CA000B003E01042208003E01D00002040206000000803F59F09F02003E013F032C0058
:20D3EA003E01000000803E597DEE0200031140410000010F010070000111AAAA0000000FD5
:20D40A0000007000001125EC0200140F2D3802001C0F00000000000F09000000680F020028
:20D42A0000001E0E000000803F59000000803E5900000000000F001002003E01E300020042
:20D44A00000601000000000F001002003E0139010200000600000000000F24EC02000011E7
:20D46A002C38020000130180020000118A8C02000010001002003E012101020000068B8CDB
:20D48A0002000010001002003E01FA00020000062F8C020000102C8C020004100410080066
:20D4AA003E01F40002000206DB0FC940040F042008003E012F8C02000011F9160204BE060D
:20D4CA002F8C02000011000000000000B78C02000110010013003E010180020000118C8C1F
:20D4EA0002000010001002003E010B0102000006308C020000102D8C0200041004100800F2
:02D50A003E01E0
:00000001FF
